:020000040800F2
:10000000681B00207D020008E94B0008A545000898
:1000100000000000000000000000000000000000E0
:100020000000000000000000000000008D560008E5
:100030000000000000000000355200089156000842
:100040008F0200088F0200088F0200088F0200084C
:100050008F0200088F0200088F0200088F0200083C
:100060008F0200088F0200088F0200088F0200082C
:100070008F0200088F0200088F0200085157000805
:100080008F0200088F0200088F0200088F0200080C
:100090008F0200088F0200088F0200088F020008FC
:1000A0008F0200088F0200088F0200088F020008EC
:1000B0008F0200088F0200088F020008D580000818
:1000C00000F002F800F0AFF80CA030C8083824188F
:1000D0002D18A246671EAB4654465D46AC4201D180
:1000E00000F0A1F87E460F3E0FCCB6460126334203
:1000F00000D0FB1AA246AB46334318479C9600003B
:10010000BC9600000023002400250026103A01D3ED
:1001100078C1FBD8520700D330C100D50B607047BF
:1001200010B56E2902D100F009FB10BD702902D173
:1001300000F04BFC10BD662902D109F035F910BD65
:10014000652902D109F030F910BD672902D109F003
:100150002BF910BD612902D109F02EF910BD0368F9
:100160001B0A01D380231943692902D100F0B0FA98
:1001700010BD642902D100F0ABFA10BD752902D17F
:1001800000F0A6FA10BD6F2902D100F0C9FB10BD26
:10019000782902D100F006FC10BDE92902D100F057
:1001A00065FB10BDE42902D100F060FB10BDF5290C
:1001B00002D100F05BFB10BDEF2902D100F0BCFBC7
:1001C00010BDF82902D100F0FBFB10BD0368DB096C
:1001D00001D380231943632902D101F0FEF810BD39
:1001E000732902D101F001F910BDE32902D101F018
:1001F0000BF910BDF32902D101F00EF910BD00205A
:1002000010BD1FB501F06EF904000020002109F0B7
:10021000B5F8401C60600020002109F099F8E0600A
:100220001FBD10B510BD01F036F91146FFF7E9FF0B
:1002300008F062FB01F066FC03B4FFF7F2FF03BCB9
:1002400000F0AEFC70B505460C46164602E00FCC39
:100250000FC5103E102EFAD2082E02D303CC03C5D0
:10026000083E042E07D301CC01C5361F03E02178D8
:100270002970641C6D1C761EF9D270BD074880473A
:1002800007480047FEE7FEE7FEE7FEE7FEE7FEE77A
:1002900004480549054A064B704700004D570008C1
:1002A000C100000868150020681B002068170020A6
:1002B00068170020FEB5054610460C46184373D05B
:1002C000AE468C460020AD1A01469C4167D3664677
:1002D000002701243D46B61A9D4102D313463A46F3
:1002E0002124654676462F04360C3E432D0CB61A63
:1002F0009D4104D3150C1B042B4312041034654696
:1003000076462F06360A3E432D0AB61A9D4104D37F
:10031000150E1B022B4312020834654676462F0742
:1003200036093E432D09B61A9D4104D3150F1B0112
:100330002B431201241D65467646AF07B6083E439F
:10034000AD08B61A9D4104D3950F9B002B43920034
:10035000A41C65467646EF0776083E436D08B61A3C
:100360009D411AD392185B41641C16E00018764632
:1003700065464941B71A9D410191009009D36046F5
:10038000B11A98418E468446009801990025401C78
:100390006941DD0752082A435B08641EE6D57246B0
:1003A000634603B0F0BDFFE700200146C046C046EB
:1003B0002A462346F5E700007CB51D4616460C008C
:1003C000009001D00019401E084B7B442A46694624
:1003D0000190304600F0CBF9002C054603D0694669
:1003E000002000F0D7F928467CBD0000D1030000B2
:1003F0000EB5044615460E4612A000F0C1FB20467D
:1004000000F0BEFB15A000F0BBFB304600F0B8FBCF
:1004100014A000F0B5FB6C460020E0720A20A07228
:100420000A3407E00A21284600F04AF83031054630
:10043000641E2170002DF5DC204600F0A1FB00F0C9
:1004400095FB00002A2A2A20617373657274696F14
:100450006E206661696C65643A2000002C20666934
:100460006C6520002C206C696E65200001E004C0E2
:10047000091F0429FBD28B0701D50280801CC90704
:1004800000D00270704700290BD0C30702D0027061
:10049000401C491E022904D3830702D50280801C18
:1004A000891EE3E70022EEE70022DFE700220309CE
:1004B0008B422CD3030A8B4211D300239C464EE07F
:1004C00003460B433CD4002243088B4231D303093B
:1004D0008B421CD3030A8B4201D394463FE0C309ED
:1004E0008B4201D3CB01C01A524183098B4201D305
:1004F0008B01C01A524143098B4201D34B01C01AF0
:10050000524103098B4201D30B01C01A5241C30867
:100510008B4201D3CB00C01A524183088B4201D3D6
:100520008B00C01A524143088B4201D34B00C01AC2
:100530005241411A00D201465241104670475DE0D7
:10054000CA0F00D04942031000D34042534000225A
:100550009C4603098B422DD3030A8B4212D3FC2203
:10056000890112BA030A8B420CD3890192118B4282
:1005700008D3890192118B4204D389013AD0921198
:1005800000E08909C3098B4201D3CB01C01A524153
:1005900083098B4201D38B01C01A524143098B421C
:1005A00001D34B01C01A524103098B4201D30B0105
:1005B000C01A5241C3088B4201D3CB00C01A52412A
:1005C00083088B4201D38B00C01A5241D9D2430811
:1005D0008B4201D34B00C01A5241411A00D201464E
:1005E000634652415B10104601D34042002B00D5B8
:1005F0004942704763465B1000D3404201B500207A
:10060000C046C04602BD70477047704770B504468B
:1006100085690068C10601D5302600E02026C007A4
:1006200007D070BD62683046A1689047206A401CC0
:1006300020626D1EF6D570BD70B5044685690078E0
:10064000C00707D170BD6268A16820209047206A6A
:10065000401C20626D1EF6D570BD09684A0501D5A3
:1006600040B27047C905FCD500B2704709684A0519
:1006700001D5C0B27047C905FCD580B2704770B5CE
:100680000C460546012A05D02878800600D5EA697F
:10069000002302E0012305E05B1C934202D2E05CF0
:1006A0000028F9D1A869E618C01AA861286AC018FC
:1006B00028622846FFF7AAFF04E06A682078A96844
:1006C000641C9047B442F8D32846FFF7B5FF70BDCD
:1006D000F7B5002575291068009914A611D0FFF709
:1006E000BCFF002802DA404211A608E00099096820
:1006F0008A0701D50FA602E0490704D50EA60125F9
:1007000001E0FFF7B3FF009F0024243704E000F06E
:10071000ADFE30313955641C0028F8D12B463246E5
:100720002146009800F07FFAFEBD000000000000A6
:100730002D0000002B00000020000000116802685E
:10074000006A530501D5087009E0D30501D508807A
:1007500005E0130602D5C21705C100E008600120BC
:100760007047000001694A1C02610878704700B5B3
:100770008FB00291002105910549019379440391BD
:1007800011460490684600F02DF90FB000BD00003E
:10079000E5FFFFFF0A681070521C0A6070470CC921
:1007A00008399A4202D2531C0B6010707047000047
:1007B000F7B50446154686B02B487844002703C891
:1007C0003E460090019111E007986A467100415A37
:1007D00002A800F025FE411C07D02178890603D528
:1007E000E269391891420ED83F18761C20788006AD
:1007F00002D5E069B84206DDAE42E5DB079871003C
:10080000405A0028E0D1A069C01BA0612046FFF734
:10081000FDFE154878445A3803C800900020019125
:1008200016E041006A460798415A02A800F0F8FD18
:100830000590401C0AD0002505E0626802A8A16866
:10084000405D90476D1C05988542F6D30498401C86
:10085000B0420490E5DB206AC01920622046FFF711
:10086000EBFE09B0F0BD00004A8E0000F7B5D21DC6
:100870000025D20815A6D200F52905CA11D0002AF4
:1008800005DA00214042914111A60A4608E000998C
:1008900009688B0701D50FA602E0490701D50EA60E
:1008A00001251146009F0024243704E000F07EF962
:1008B00030323A55641C02460A43F7D12B46324681
:1008C0002146009800F0AFF9FEBD000000000000D6
:1008D0002D0000002B0000002000000070B5044631
:1008E0000021243408E05507D2086D0F30356554D7
:1008F0005D072A43DB08491C15461D43F3D10468F4
:10090000002310A2250708D5A40601D4002904D08D
:10091000C46901230CA2641EC46100F084F970BD97
:1009200010B5044621461068FFF7A0FE00230246DA
:100930002046FFF7D3FF10BDD21DD108C9000CC956
:10094000CCE700000000000030000000F8B50F46C2
:100950000188090502D5224C7C4402E0204C7C44ED
:100960000E3405460021243508E016071209360F1B
:10097000A65D6E541E0732431B09491C16461E43D2
:10098000F3D1224604780023240705D5702F06D022
:10099000002901D00223113200F045F9F8BD0123EE
:1009A0001032F9E770B504460D4621461068FFF78E
:1009B0005DFE0023024629462046FFF7C7FF70BDB3
:1009C000D21DD308DB000CCBC0E730B40368202471
:1009D0001268234303600823C36130BC0023B5E7DA
:1009E000B48C0000F3B50446002081B0206220469C
:1009F000E1688847002872D0252802D06268A16883
:100A0000ABE0594F00267F442046E1688847202804
:100A1000054608DB312D06D27819203800780028E9
:100A200001D00643F0E7B00701D50420864300203B
:100A3000E0610746A0612A2D0AD0284607F014FC81
:100A4000002827D0B8000019303D0090856119E0DA
:100A50000298BA00121902C8916102902046E1681A
:100A60008847012F054617D1E06900281FDA2020AA
:100A700086431CE000980A21806948430099401988
:100A8000303888612046E1688847054607F0ECFB6E
:100A90000028EFD1012F0AD02E2D08D12046E16881
:100AA00088470546202006437F1C022FC3DBA06930
:100AB000002803DA4042A06101200643F00701D07C
:100AC000102086436C2D0BD0682D09D04C2D3CD0C6
:100AD0006A2D38D0742D38D07A2D36D016E040E00B
:100AE000E1682F4620468847B842054609D16C2F59
:100AF00029D001208002E168064320468847054648
:100B000004E06C2F1DD0FF2001300643002D28D0BB
:100B100028464138192803D80120C0020643203551
:100B2000204626602946029A1646FFF7F9FA002861
:100B300010D001280BD0F61DF008C000083002903C
:100B400055E74020E1E78020D5E70020D3E7361DB8
:100B500002964CE762682846A1689047206A401CCC
:100B600044E7206AFEBD00002E8C000010B5002076
:100B700000F076FCFFF755FB012000F011F810BDE6
:100B800010B5044602E0641C00F004F82078002848
:100B9000F9D110BD08B5694608700320ABBE08BD89
:100BA00001491820ABBEFEE7260002000B4670B5D7
:100BB000024689078008084319469D08141AA9416E
:100BC00025090807054308092C194841250A01068B
:100BD0000D43010A2C194141200C0D0428430D0C32
:100BE00000194D41002140194D41C00869070843D3
:100BF000E908840F8D002543840024184D412419F1
:100C00006D41121BAB4107E00925ED432C11521930
:100C100063410024401C61411C460A250026551BE7
:100C2000B441F1D270BDFFB504460D4681B0243009
:100C300000902168880604D51022E0699143216064
:100C400000E00120A84201DD471B00E000270498D6
:100C5000A1697A191018081AA0612078C00602D478
:100C60002046FFF7D3FC002608E003986268A168DD
:100C7000805D9047206A401C761C20620498864262
:100C8000F3DB2078C0060AD52046FFF7BFFC06E05C
:100C90006268A16830209047206A401C2062384674
:100CA0007F1E0028F4DC07E000986268A168405DC0
:100CB0009047206A401C206228466D1E0028F3DC05
:100CC0002046FFF7B9FC2078000602D5022005B0C7
:100CD000F0BD0120FBE700007047FFB50C461E4643
:100CE0008FB003CA089009914F007D0D00D16D1E91
:100CF000002108460020C0460321099A89050840C2
:100D0000002A03DA8200801840080840800D01287C
:100D10000A9002DD0020C0430A90089807430DD0D6
:100D2000EF48F049281848430714189800281DD0A8
:100D30007542291E1DDD0A9842421BE018980128C1
:100D400002D00020302104E00020F24305E02154CD
:100D5000401CB042FBDB30460022189B002121548E
:100D60000F998B600A60486013B0F0BDBD1B6D1C0D
:100D7000DFE70A9A002900DA69420BA800F0FAFBC3
:100D80000BAB07CB03AB07C30899099800F056FCDF
:100D90006B4607C30146D4480918002D00910ADDAF
:100DA000D14903980A9A4942401803A9039068461A
:100DB00000F077FE07E003990A9A081803A9039048
:100DC000684600F036FE6B4607C30004000C03D0F3
:100DD0000020C043410800E01046189A002A03D0C2
:100DE0000022009215461EE0751E05D4FFF7DEFEB8
:100DF000303262556D1EF9D501220843079602D0A4
:100E000000227F1C04E02078302801D100227F1EC0
:100E1000002A069789D01EE0112D07DAFFF7C6FEDB
:100E2000303262556D1C02460A43F5D1084303D0A7
:100E30000098002819D00EE00021681E05E0235C10
:100E4000625C63542254401E491C8142F7DBA81B9C
:100E5000401E07950690079A18990020A0540F98F5
:100E6000079B069A81600CC07EE71126002018902F
:100E70005BE7D21DF0B50D460446D10893B0C9001A
:100E800003C90C900D9107F09DF902460D98C00F13
:100E900001D02D2007E02068810701D52B2002E03A
:100EA0004007C00F4001032A0F9001D0072A05DB3D
:100EB00003462946204600F019FB0EE12078800603
:100EC00001D5E76900E006272846652D04D066288D
:100ED00014D0672D69D12DE00020112F009001DB87
:100EE000112300E07B1C0CAA03A910A8FFF7F5FE54
:100EF0001199002610987D1C0E9142E001203B467E
:100F00000CAAC0070B900120009003A910A8FFF7BE
:100F1000E4FE119D12981099002600280E9501D12B
:100F2000781C0D18781B02D446427D1C761EE81BE7
:100F300000903AE0012F00DA01270020112F0090E5
:100F400001DD112300E03B460CAA03A910A8FFF71E
:100F5000C4FE11993D46109800260E91217809078C
:100F60000BD40E99A94200DA0D4603A9012D04DD28
:100F70004A19203AD27F302A06D0B84201DA011D40
:100F800004DA012100910FE06D1EEFE7002802DC7A
:100F900086192D1A03E0411CA94200DD0D46801B75
:100FA000401C00900120C0070B902078000705D45A
:100FB0000098A84202DB0020C04300906946002050
:100FC000C8720B98012102AF0337C907884225D0A8
:100FD000022010902B2011900B9800280BDA404231
:100FE0000B902D20119006E00B9800F03FFA303165
:100FF0007F1E0B9039701099481E00291090F3DC69
:101000000B980028F0D111987F1E387020880005B9
:1010100001D5452000E065207F1E387001A8C01B67
:10102000C01D0B900F98002800D001204119009896
:10103000C01709180B980818A169081A401EA0616A
:101040002078C00602D42046FFF7E0FA0F98002867
:1010500005D06268A1689047206A401C2062207811
:10106000C00625D52046FFF7D1FA21E0002E07DB88
:101070000E98B04204DD03A86268805DA16802E0BA
:101080006268A16830209047206A761C401C20626C
:101090000098401E002800900AD100F023FAC06892
:1010A00062680168405CA1689047206A401C206229
:1010B00028466D1E0028D9DC07E062683878A168F0
:1010C0007F1C9047206A401C20620B99481E002913
:1010D0000B90F2DC2046FFF7AFFA032044E6000055
:1010E00001FCFFFF104D0000E1DFFFFFD21DF0B556
:1010F00004460D46D0088DB0C000466807683146EA
:10110000384607F05FF80246F00F01D02D2307E0C4
:101110002068810701D52B2302E04007C00F43015F
:101120006846002B037001D0012000E00020032A54
:101130000A9001D0072A04DB2946204600F0D6F9A0
:101140002DE12078800601D40D2500E0E5697000CE
:10115000400D0D2D01904BDA300D00210B9008460B
:101160000020C046032189050840002E05DA8200D0
:101170008018C20F1018401008408015012801DDAA
:101180000020C043A9000023182906D39C460A4624
:101190000123183A1B07D34003E001221205CA407D
:1011A00094460C31202902D33A46203900E03246D9
:1011B0008A40002802DD002A06D119E0002817D154
:1011C0000121C9078A4213D3194663467F185E413D
:1011D000002806D10120C007824202D10846874379
:1011E0009E430B98310D814202D00198401C019022
:1011F0002088000502D57149794402E06F4979449D
:1012000019396B460A9830221A540A980A7C401CF5
:101210001A54401C0A900198002801DC302000E09C
:1012200031201872019A0120002A02D0644BD21892
:1012300004E072003A4302D0614A521C0192002D30
:1012400002DC2278120703D56A462E205072022053
:101250000022864694460CE032033601120F6D1EC2
:101260008B5C02AA13546246521C401C9446052A09
:1012700001DA002DF0DC002202AE08E03B0F3F0156
:10128000CB5C521C6D1E3354401C082A01DA002D21
:10129000F4DC23689A0601D511E0401E704504DD98
:1012A0003218203AD27F302AF7D0002807DD3218D2
:1012B000203AD27F2E2A02D11A0700D4401E002DD8
:1012C00003DD3E223254401C6D1E497C315401998D
:1012D000401C002906DA2D21471C31540198404258
:1012E000019003E02B21471C315401987D21C90056
:1012F000884206DBFFF7E4F83030F0557F1C01919F
:1013000001E0642808DB01986421FFF7D9F8303048
:10131000F0557F1C019101E00A2806DB01980A21A3
:10132000FFF7CEF83030F0557F1C01980A21FFF707
:10133000C7F83031F1550A98A1697F1C7A19101845
:10134000081AA0612078C00602D42046FFF75EF993
:10135000216A6E460A980818206204E062683078B4
:10136000A168761C90470A98401E0A90401CF5D14F
:101370002078C00602D52046FFF748F902AE09E002
:101380003078761C3E280DD06268A1689047206AAC
:10139000401C20627F1EF3D22046FFF74DF90DB0AE
:1013A0000320F0BD206A4019206203E06268A16852
:1013B000302090476D1EEDD3F8E7000060840000F8
:1013C00001FCFFFF10B54369002B02D0C046C046A8
:1013D00001E0FFF754F9012010BD127801462431D5
:1013E0000A7000224A700122ECE711680022D24301
:1013F000E8E710B54369002B02D0C046C04601E0C3
:10140000FFF7D6F9012010BD1288014624318284ED
:101410000022C2840122ECE711680022D243E8E7EF
:1014200070B516460C46054600F054F80368FF20D8
:101430000230C05C012807D0FF2C0ED8185D0028B0
:101440000BD001202C7070BDFF333246214608338B
:101450001868C3182846984770BD0020C04370BD67
:1014600010B500F05DFB00F055FB10BD0146800893
:10147000081A02091018020A1018020C1018C008E5
:10148000820012185200891A01E0401C0A390A2908
:10149000FBD270477047754600F05AFBAE46050018
:1014A00069465346C008C000854618B020B5FEF70F
:1014B000EFFE60BC00274908B6460026C0C5C0C57F
:1014C000C0C5C0C5C0C5C0C5C0C5C0C5403D490038
:1014D0008D46704710B500F005F8001D10BD00BF27
:1014E0009D7E00000048704728150020F8B51F4673
:1014F000044601230068DB02032601461840072A40
:1015000005DB002801D017A506E017A504E0002898
:1015100001D016A500E016A5102081432160A06926
:10152000C01E002FA06101D0401EA0612046FFF721
:101530006DF8002F09D038466268A1689047206A8C
:10154000401C2062C01C206206E0206AFAE7626844
:101550002878A1686D1C9047761EF8D22046FFF7C8
:101560006BF8F8BD4E414E006E616E00494E46006C
:10157000696E6600F7B516468AB02F4878446C4607
:1015800003467C33C06F5A689B680DC42A48784470
:10159000763003AC0DC80DC43720C00108183721C0
:1015A0001B30FEF78DFF05460C46803D1B3C02D5E7
:1015B0006442012000E00020002709900FE0E007CE
:1015C0000BD00C201C497843794432464C394118E1
:1015D000684600F02EFA6B4607C364107F1C002C8F
:1015E000EDD1154F7F442C3F15E0E80711D02001C5
:1015F000C0190EC80691089307920068F04201D105
:1016000098190890324606A903A800F012FA03AB15
:1016100007C36D10641C002DE7D132466946099856
:10162000002803A802D000F03CFA01E000F001FA23
:101630000A9B07C30DB0F0BDF080000003464000D8
:101640000A4610B5400D0BD00121C9070F24A40292
:1016500000191C0364082143540D2143D20207E002
:1016600000210120F2E7D40F490021435200401E1F
:101670000029F8DADB0FDB07184310BDFFB50D4674
:10168000144685B04868516806F076FD00910190D7
:10169000A868A16806F070FD02910390A8686168CF
:1016A00006F06AFD029A12188242029201D20120CB
:1016B00000E00020019A0B18D2180028019202D0F5
:1016C0008A4202D903E08A4201D2012000E00020D0
:1016D0000099081800906868A16806F04DFD029A0C
:1016E00012188242029201D2012000E00020019AE9
:1016F0000B18D2180028019202D08A4202D903E0C6
:101700008A4201D2012000E00020009908180090D0
:101710002868216840004900400849084018F549F8
:10172000471814E001994000C90F08430090019840
:1017300002994000C90F08430190029803994000A4
:10174000C90F08430290039840007F1E0390009841
:101750000028E7DA0898002801D0E74E00E00026CC
:10176000B74228DAF71BF806C00E15D0029B2021DD
:10177000091A039A8B401A430392029A019BC240B2
:101780008B401A430292019A009BC2408B40009901
:101790001A430192C14000917A110BD06B4603208D
:1017A000811A01D5002101E0890059588700401EA7
:1017B000D951F5D5374603980299002800D0012069
:1017C000014308980291002808460CD0002800D058
:1017D00001200199019A490508430121D20AC90251
:1017E000D202019200E001210E9B0122D207012BBF
:1017F00002D0002B03D013E0002807D116E090425E
:1018000004D890420CD1019B0B4209D0019B59187E
:10181000019105D10099491C009101D17F1C0092D2
:10182000002803D0102108460020C04628682168FF
:10183000019B009A4840C10F0598C90739430EC063
:1018400009B0F0BDFFB587B0099A089808995368A8
:10185000926840688968964600220393174694462A
:10186000089A12685300099A5B08126852005208DD
:101870009A1AA24BD4180A9A002A01D0352200E005
:10188000402206920022012315460492DB070593AD
:1018900024E0002D05D175460346039E4D1BB34140
:1018A00009D375466646039B491B049D9841059BD9
:1018B0007519AC465F4163463B4308D0059B049EC7
:1018C000DD0776082E435B080496059301E0521E5F
:1018D000641EC50FED0749184041521C069B9A42F1
:1018E000D7DB002D04D17546039A6B1A824101D2D1
:1018F00003200CE0039A0B466B404240134303D095
:10190000014303D0012002E0022000E000206146F4
:1019100001910021009702910A99002905D06146A2
:1019200040020143744B019102E0800700230290C2
:101930009C423ADA1A1BD006C00E15D0029D202117
:10194000019C091AC5408C402543029C8C4000D064
:1019500001242543019C02953D46C4408D403946F3
:101960002C43C1400194009154111DD06D460221B9
:10197000002202290CD10320001B07E0002804DB11
:101980008600AE59002E00D00122401C0328F5DB52
:10199000081B02D588002A5004E080002858104314
:1019A0008A00A850491EE3D51C460A9800280298D0
:1019B0000CD0002800D001200199019A4905084364
:1019C0000121D20AC902D202019200E00121109B3A
:1019D0000122D207012B02D0002B03D013E00028F4
:1019E00007D116E0904204D890420CD1019B0B42E3
:1019F00009D0019B5918019105D10099491C00910A
:101A000001D1641C0092002803D010210846002058
:101A1000C04608980999019A0068096848400099E9
:101A2000C30F0798DB0723430360826041600BB05C
:101A3000F0BD1FB5002300920A46014601A8FFF73A
:101A40001DFE01AB07CB04B010BDF0B585B001237E
:101A500000920A46014601A8FFF710FE01990F22E5
:101A600002989202CF0F4900039E49088C1AFF0783
:101A70000021002800DB0C46450021486D08844207
:101A800006D30D460E460446102108460020C046E7
:101A90002005E90A084369053843F20A05B01143F5
:101AA000F0BD1FB5002300920A46014601A8FFF7CA
:101AB000C9FE01AB07CBC6E71FB5012300920A465A
:101AC000014601A8FFF7BEFE01AB0F2407CBA4021D
:101AD000C30F4000DB074008001B002900DB00208B
:101AE000490000054908CC0A204349051843D20A99
:101AF0001143A8E702C0FFFF013C0000FF3F0000C8
:101B0000FF07000010B50446C046C0462046FEF759
:101B100093FB10BD10B5002801D0FFF741F810BDB0
:101B200010B5002102A000F017F8012010BD000040
:101B3000534947414252543A2041626E6F726D617F
:101B40006C207465726D696E6174696F6E0000005F
:101B5000004870470815002070B505460C460A205D
:101B600000E06D1CFFF716F8002D06D0287800283D
:101B7000F7D102E0641CFFF70DF8002C02D02078AA
:101B80000028F7D10A20FFF705F870BD024670B5AE
:101B90000A4392072AD11E4DEE0104C808C9541BFE
:101BA0009443344017D0D0B2D9B2401A2106014331
:101BB00010D190B299B2401A210401430AD1100207
:101BC0001902000A090A401A2102014302D1100E2B
:101BD000190E401A70BD9A42DFD010BA19BA884265
:101BE00001D9012070BD0020C04370BD02780B7880
:101BF000401C491C002A09D09A4207D102780B7870
:101C0000401C491C002A01D09A42EFD0D01A70BD66
:101C10000101010170B58C180578401C6B075B0F42
:101C200001D10378401C2A1106D10278401C03E040
:101C30000678401C0E70491C5B1EF9D12B0705D499
:101C40000023521E0DD40B70491CFAE70378401C88
:101C5000CB1A921C03E01D780D70491C5B1C521EB0
:101C6000F9D5A142D8D3002070BD0346042B16D06D
:101C700008DC002B0FD0012B0ED0022B0DD0032B34
:101C800012D10BE0202B0BD0212B0AD0222B09D014
:101C9000232B09D107E008E007E006E005E004E0B7
:101CA00003E002E001E000E000BF00BF0020704759
:101CB0000020704710B500220449054803F03FFF9B
:101CC0000449034803F031FF002010BDD00B002071
:101CD0000C030020D007002070B504460E460948CA
:101CE000856B2146084803F020FF074803F0EFFE0C
:101CF000832080004059054908600120044908708C
:101D0000002070BD8C0500200C0300207C0000200A
:101D100078000020F8B504460D4600260948876B78
:101D200085208000C059002801D00120F8BD2A4636
:101D30002146054803F003FF034803F097FF0646DA
:101D40003046F3E78C0500200C03002072B600BF7C
:101D5000FEE70000FEB504460025324E3746304609
:101D60000190009000F0FAF80443E6B2FF20000270
:101D70002040070AFF2000042040000C0190200EA4
:101D80000090294800F0A4F90546002D48D12749C4
:101D9000C86100F01BFA0546002D41D124480069B6
:101DA0001021084322490861FF2E08D021480089EC
:101DB0003040204908811C4800F08AF90546002D72
:101DC0000AD1FF2F08D01B48408938401949488163
:101DD000154800F07DF90546002D0CD10198FF282B
:101DE00009D01448808901990840124988810E4819
:101DF00000F06EF90546002D0CD10098FF2809D09F
:101E00000C48C089009908400A49C881064800F07A
:101E10005FF90546064800691021884304490861B6
:101E20002846FEBDFFFF000050C30000E81400205C
:101E30000020024000F8FF1FFEB504460025334E87
:101E4000374630460190009000F088F8C0432043A8
:101E5000C443E6B2FF2000022040070AFF2000042E
:101E60002040000C0190200E0090294800F030F92D
:101E70000546002D48D12749C86100F0A7F905465D
:101E8000002D41D1244800691021084322490861EE
:101E9000FF2E08D0214800893040204908811C4885
:101EA00000F016F90546002D0AD1FF2F08D01B4877
:101EB0004089384019494881154800F009F905461C
:101EC000002D0CD10198FF2809D014488089019970
:101ED0000840124988810E4800F0FAF80546002DA6
:101EE0000CD10098FF2809D00C48C08900990840FF
:101EF0000A49C881064800F0EBF805460648006923
:101F000010218843044908612846FEBDFFFF0000F8
:101F100050C30000E81400200020024000F8FF1F1A
:101F20000848C069062210400146002901D1AA20B4
:101F3000704704200840042801D1CC20F8E7BB20DA
:101F4000F6E70000002002400348C069772109023B
:101F50000840000A70470000002002400148006A63
:101F6000704700000020024070B504460D4601266F
:101F70000D4800F0ADF80646002E12D10B49C8619D
:101F80000B4800691021084309490861258006486B
:101F900000F09EF80646064800691021884304496F
:101FA0000861304670BD000050C30000E8140020F6
:101FB0000020024070B5054600241A4800F088F859
:101FC0000446002C2BD11849C8611848006920210B
:101FD000084316490861084600694021084313492F
:101FE0000861104800F074F8044610480069202188
:101FF00088430E490861002C11D108460069102160
:1020000008430A4908610A480580064800F060F85C
:1020100004460648006910218843044908612046A7
:1020200070BD000050C30000E814002000200240F2
:1020300000F8FF1F70B5054600240F4800F048F86F
:102040000446002C15D10D49C8610D4800691021C6
:1020500008430B490861882028430A4948800648FC
:1020600000F036F804460648006910218843044908
:102070000861204670BD000050C30000E814002035
:102080000020024000F8FF1F00200F49C9681022FD
:102090001140102907D10D49C969022211430B4A89
:1020A000D161102108430849C9680422114004295C
:1020B00007D10649C96901221143044AD1610421AB
:1020C00008430149C860704700200240E81400201E
:1020D00070B5044600F088FA05460BE0601C002845
:1020E00008D0002C04D000F07FFA401BA04201D998
:1020F000032070BD0F48C068C007C00F0028EDD195
:102100000C48C06820210840202801D10949C86036
:102110000848C06810210840102805D00548C0684C
:1021200004210840042803D1FFF7AEFF0120E0E7B7
:102130000020DEE7002002400148006870470000F0
:1021400000F8010870B50948C46A056B466BA4190C
:10215000002C0AD008220649204602F0EBFB04229C
:1021600003491031284602F0E5FB70BD80F7FF1FE0
:102170005E00002030B50246134600200BE004123A
:102180001D786C402406E40D044D2C5B05026C4068
:10219000A0B25B1C491E0029F1D130BDC8930008D4
:1021A00070B5044600F020FA06462546681C002853
:1021B00002D0054800782D1800BF00F015FA801BEA
:1021C000A842FAD370BD00009800002070B5AA257F
:1021D0000124FFF7A5FEC5B21248FFF779FF0446B8
:1021E000002C1DD11049C861104800692021084306
:1021F0000E49086108460069402108430B490861FF
:102200000848FFF765FF0446084800692021884315
:1022100006490861002C03D12846FFF7CBFE04468F
:10222000204670BD50C30000E8140020002002408A
:1022300010B5044607202060FFF790FEA060FFF76E
:102240006FFE2073FFF780FE607310BD70B504460B
:10225000012500BF3048007E012801D1022070BD59
:1022600001202D49087600BF2078C007C00F002844
:1022700014D06068012804D1A068FFF7DDFD054691
:1022800003E0A068FFF766FD0546002D06D000BFFD
:1022900000202149087600BF2846E0E70221206897
:1022A000084002280CD1207BFFF784FE0546002D54
:1022B00006D000BF00201849087600BF2846CEE7A8
:1022C00004212068084004280CD1607BFFF7B2FE8F
:1022D0000546002D06D000BF00200F49087600BF3C
:1022E0002846BCE708212068084008280DD1217D38
:1022F0002069FFF739FE0546002D06D000BF0020FB
:102300000549087600BF2846A9E700BF002002491A
:10231000087600BF2846A2E7E814002003480069B9
:1023200080210843014908610020704700200240D5
:1023300010B50548006901214903084302490861B5
:102340000248FFF7C5FE10BD0020024050C3000048
:1023500004480069012149028843024908610020BC
:10236000704700000020024008480069012149022E
:102370000840002805D1064804498860054888605F
:1023800001E0012070470020FCE70000002002402F
:1023900023016745AB89EFCD0020094909698022F7
:1023A000114000290BD00749054A51600649516088
:1023B0001146096980221140002900D00120704790
:1023C0000020024023016745AB89EFCD78B5034675
:1023D0000A460021E4E001268E4014683440002CB7
:1023E0007ED01579AD07AD0F012D04D01579AD075D
:1023F000AD0F022D18D198684E000325B540064652
:10240000AE4330464E00D568B540284398605868C2
:1024100001258D400646AE433046102655683540AE
:102420002D098D40284358601579AD07AD0F032D58
:102430000BD0D8684E000325B5400646AE43304663
:102440004E009568B5402843D8601579AD07AD0FAB
:10245000022D15D1CD08AE001D462035A8594D07D7
:10246000EE0E0F25B5400646AE4330464E07F60E3B
:102470001569B5402843CD08AD001E462036705181
:1024800018684E000325B5400646AE433046157920
:10249000AD07AD0F4E00B540284318600326360443
:1024A00055683540002D7AD000BF404DAD690126FA
:1024B00035433E4EB5613546AD69ED07ED0F0095EC
:1024C00000BF00BF3A4D8E08B600A8598D072E0FE9
:1024D0000F25B5400646AE4330460925ED0600E01F
:1024E0005DE0AB4201D1002514E0324DAB4201D199
:1024F00001250FE0304DAB4201D102250AE02F4DFE
:10250000AB4201D1032505E02D4DAB4201D104259D
:1025100000E005258E07360FB5402843244D8E0870
:10252000B600A851274DA8680546A54328460126B0
:10253000360555683540002D02D00546254328460E
:10254000204DA860E8680546A54328460126760583
:1025500055683540002D02D0054625432846194DC3
:10256000E86068680546A543284601267604556854
:102570003540002D02D0054625432846114D6860A0
:1025800028680546A5432846012636045568354087
:10259000002D02D00546254328460A4D2860491CD7
:1025A0001568CD40002D00D015E778BD0010024021
:1025B000080001400004004800080048000C0048E2
:1025C0000010004800040140024613690B40002B34
:1025D00001D0012000E000207047002A01D0816175
:1025E00000E0816270470000014800687047000009
:1025F0009000002002464120805C20282FD100BF9F
:102600004020805C012801D1022070470123402036
:10261000835400BF2423412083541068006840087D
:102620004000136818601068006801231B0398437A
:102630001368186010680068084313681860106811
:102640000068012318431368186020234120835435
:1026500000BF00234020835400BF0020D5E70220A4
:10266000D3E710B502460B464120805C20282ED1CE
:1026700000BF4020805C012801D1022010BD012450
:102680004020845400BF24244120845410680068F2
:102690004008400014682060106801680F2424027C
:1026A0000846A04301461802014310680160106803
:1026B00000680124204314682060202441208454B1
:1026C00000BF00244020845400BF0020D6E7022031
:1026D000D4E7000010B50446002C01D1012010BD44
:1026E0004120005D002805D10021402001552046F1
:1026F00000F00CFA242141200155206800684008B0
:102700004000216808600F2109066068884321683D
:102710000861206880680121C903884321688860B6
:10272000E068012806D10121C903A0680843216897
:10273000886005E021218902A0680843216888603B
:10274000E068022802D18002216848602068406861
:1027500014490843216848602068C0680121C90302
:1027600088432168C860616920690843A16909023A
:1027700008432168C860216AE0690843216808604D
:102780002068006801210843216808600020606417
:1027900020214120015500202063002142200155C5
:1027A00000209CE700800002FFB585B004460F467C
:1027B0001E46002004904120005D20287ED1206824
:1027C00080690121C9030840C00B002802D0022003
:1027D00009B0F0BD00BF4020005D012801D10220FA
:1027E000F6E701214020015500BF24214120015579
:1027F0000020606400BFE068012809D1B805800DA1
:1028000001214903401809034018C91388430AE00D
:10281000B805800D0121C90240188900401809033C
:102820004018C913884321684860FFF7DDFE05465C
:102830002068806920210840400903902068806951
:10284000102108400009029022E0701C002813D0DB
:10285000FFF7CAFE401BB04201D8002E0CD1202148
:1028600041200155606C0843606400BF0021402096
:10287000015500BF0120ABE7206880692021084096
:1028800040090390206880691021084000090290E7
:102890000398002802D102980028D6D020688069C9
:1028A000102108400009002819D1334600222021B8
:1028B0002046009501F09EFF002800E04EE001D088
:1028C000012085E720202168C86120214120015591
:1028D00000BF00214020015500BF002078E73346AB
:1028E000002220212046009501F084FF002801D01D
:1028F00001206DE710202168C86120202168C8618F
:1029000004990798814214D1206840680121890305
:102910000843216848603346002220212046009564
:1029200001F068FF002801D0012051E72020216834
:10293000C8610498401C049004990798814200D211
:1029400059E7202141200155606C0843606400BFB5
:1029500000214020015500BF012039E7022037E760
:10296000FFB583B004460C9F0E9E4120005D2028D9
:102970007ED1002F02D00D98002805D10120400201
:102980006064012007B0F0BD00BF4020005D012859
:1029900001D10220F6E701214020015500BFFFF7D9
:1029A00023FE054619230122D1032046009501F09C
:1029B00021FF002801D00120E4E722214120015518
:1029C0004021422001550020606467620D986085B7
:1029D0000020606300960195204604A90EC901F00D
:1029E000ABFE002806D000BF00214020015500BFEB
:1029F0000120C7E7608DFF280CD9FF2020854148C2
:102A00000090208DC2B201231B062046049901F0DC
:102A1000D3FE0BE0608D20853A480090208DC2B235
:102A200001235B062046049901F0C6FE00BF334631
:102A3000002204212046009501F0DCFE002801D090
:102A400001209FE72068406A616A0870606A401C44
:102A50006062208D401E2085608D401E6085608DE7
:102A600000282BD0208D002828D13346002200E0FA
:102A700045E080212046009501F0BCFE002801D0F1
:102A800001207FE7608DFF280CD9FF2020850020E2
:102A90000090208DC2B201231B062046049901F04C
:102AA0008BFE0BE0608D208500200090208DC2B24F
:102AB00001235B062046049901F07EFE608D00280C
:102AC000B5D12A463146204601F0CAFE002801D081
:102AD000012057E720202168C861206840680A4922
:102AE00008402168486020214120015500214220F2
:102AF000015500BF4020015500BF002042E70220E1
:102B000040E700000024008000E800FE10B586B019
:102B10000446142101A8FDF7C7FC1A492068884221
:102B20002DD100BF18484069012189040843164986
:102B3000486108464069012189040840009000BFAF
:102B400000BFC020019012200290002003900320BB
:102B500004900120059001A90C48FFF737FC00BF45
:102B60000948C0690121490508430749C861084669
:102B7000C069012149050840009000BF00BF06B0B0
:102B800010BD000000540040001002400004004846
:102B900003480068034909784018014908607047F4
:102BA000900000209800002010B506480068102111
:102BB000084304490860032000F006F800F02EF8EE
:102BC000002010BD0020024070B504461048017876
:102BD0007D20C000FDF76AFC064631460D480068BE
:102BE000FDF764FC054601F0C1FC002801D001207E
:102BF00070BD042C07D200222146501E00F03CF884
:102C00000548046001E00120F2E70020F0E7000041
:102C1000980000209C0000209400002008B500BF10
:102C20000D488069012108430B4988610846806985
:102C3000C007C00F009000BF00BF00BF0846C069BA
:102C4000090408430449C8610846C06909040840EA
:102C5000009000BF00BF08BD0010024001460029DF
:102C600005DBCB06DB0E01229A40024B1A6000BF47
:102C70007047000000E100E070B504460D461646BE
:102C80002946204605F0B4FA70BD01460A680120C5
:102C90000523DB01CB189866002017235B01CB18B6
:102CA00018705420805A01231843542398525420FA
:102CB000805A0223184354239852002070477047CB
:102CC00070B505460C4680202040802806D160075C
:102CD000400F28267043AE19811905E02820604373
:102CE0002E46FF3669368119002A03D10020087369
:102CF000CB8004E0012008730B81180C4881002070
:102D000070BD70B504460D4628216943234628331B
:102D1000C9184A690521C9016118086F294603F0DD
:102D200008FB70BD70B504460D4628216943234653
:102D3000FF336933C9184A690521C9016118086F51
:102D4000294603F091FB70BD70B504460E46802005
:102D50003040802808D17007400F2821484361186F
:102D600045180120687009E07007400F282148438A
:102D70002146FF3169314518002068707007400F07
:102D8000287000BF152040012018007A012801D1C9
:102D9000022070BD0120152149016118087200BF91
:102DA0002946206804F09AFA00BF00201521490145
:102DB0006118087200BF00BFEBE770B504460E460D
:102DC0003007000F6168884201D9012070BD802062
:102DD0003040802808D17007400F282148436118EF
:102DE00045180120687009E07007400F282148430A
:102DF0002146FF3169314518002068700020A87015
:102E00007007400F287000BF152040012018007A7D
:102E1000012801D10220D9E70120152149016118BB
:102E2000087200BF2946206804F0AEFB00BF0020F6
:102E3000152149016118087200BF00BFC6E70000F4
:102E4000F8B505460C461746012080033840002897
:102E50004ED028684030008A2178C9004018801C74
:102E60000122920229688918405A8605B60DA06988
:102E7000B04203D3A069801BA06101E00020A061E3
:102E8000A069002813D100BF227892002968895ACE
:102E90003F4A114008460121490348408900014347
:102EA0008022114323789B002A68D15200BF402022
:102EB0003840002813D000BF00BF22789200296854
:102EC000895A344A114008460121C9030143C022EE
:102ED000114323789B002A68D15200BF00BF002E07
:102EE00054D0228961693346286805F0FFF84DE027
:102EF00028684030008A2178C9004018801D0122CE
:102F0000920229688918405A8605B60DA069B04218
:102F100003D3A069801BA06101E00020A061A0692B
:102F2000002813D100BF227892002968895A184AD4
:102F3000114008460121490348408900014380228D
:102F4000114323789B002A68D15200BF40203840AB
:102F5000002813D100BF00BF227892002968895A47
:102F60000C4A114008460121C9030143C022114304
:102F700023789B002A68D15200BF00BF002E05D0E5
:102F8000628961693346286805F0B0F83046F8BDBB
:102F90008FBF00008F8F0000F7B584B005460C4648
:102FA00040210698084000286FD028684030008AE9
:102FB0002178C9004018801C0122920229688918D2
:102FC000405A8705BF0DA069B84203D9A069C01B4C
:102FD000A06101E00020A061A06900287ED100BFAF
:102FE000607800281BD100BF29680391296840310F
:102FF0000A8A0399511803912178C900891C012379
:103000009B02039AD218881800BF01888905890D90
:10301000018001885A011143018000BF12E06078ED
:1030200001280FD100BF28682A684032128A101880
:103030002278D200921C01239B02C318D1180022CF
:103040000A8000BF00BF00BF286803906078002896
:103050001CD100BF29680191296840310A8A019971
:10306000511801912178C900891D01239B02019A01
:10307000D218881800BF01888905890D0180018850
:103080005A011143018000BF15E0D8E060780128A3
:1030900011D128684030018A0398081803902078DD
:1030A000C000801D012292020399891840180290E5
:1030B00000210298018000BF21782846FFF721FEF9
:1030C0000121890306980840002815D000BF00BFE1
:1030D000227892002968895AFC4A00E00DE01140EC
:1030E00008460121C90301438122D20111432378FB
:1030F0009B002A68D15200BFF2E1012189030698A2
:103100000840002814D000BF00BF22789200296830
:10311000895AEE4A114008460121C9030143812220
:10312000D201114323789B002A68D15200BF00BF0F
:103130002420005D0128DFD16069C0196061E06969
:10314000C019E0612169206A884204D32669206A97
:10315000801B20620DE0206A002804D13E46002139
:103160002420015505E0002124200155266A002075
:10317000206200BF6078002846D100BF2968039113
:10318000296840310A8A0399511803912178C900AE
:10319000891C01239B02039AD218881800BF01885A
:1031A0008905890D01803E2E13D900BF7109029156
:1031B000F106C90E002902D10299491E0291018827
:1031C000029A92020123DB031A4392B21143018057
:1031D00018E0002E05D101880122D203114301809D
:1031E00010E000BF71080291F107C90F002902D059
:1031F0000299491C02910188029A9206120C11430D
:10320000018000BF00BF11E0607801280ED100BF2F
:1032100028682A684032128A10182278D200921C3C
:1032200001239B02C318D1180E8000BF00BFB3B2A8
:10323000228961692868039004F080FF50E12868C2
:103240004030008A2178C9004018801D0122920276
:1032500029688918405A8705BF0DA069B84203D371
:10326000A069C01BA06101E00020A061A069002846
:103270007ED100BF607800281BD100BF2968039170
:10328000296840310A8A0399511803912178C900AD
:10329000891C01239B02039AD218881800BF018859
:1032A0008905890D018001885A011143018000BF01
:1032B00012E0607801280FD100BF28682A684032E8
:1032C000128A10182278D200921C01239B02C31884
:1032D000D11800220A8000BF00BF00BF28680390F9
:1032E000607800281BD100BF29680191296840310E
:1032F0000A8A0199511801912178C900891D012379
:103300009B02019AD218881800BF01888905890D8F
:10331000018001885A011143018000BF14E06078E8
:10332000012811D128684030018A039808180390B9
:103330002078C000801D012292020399891840184C
:10334000029000210298018000BF21782846FFF7F3
:10335000D8FC0121890306980840002815D100BF38
:1033600000BF227892002968895A584A114000E02B
:103370000CE008460121C90301438122D201114317
:1033800023789B002A68D15200BFA9E0012189035C
:1033900006980840002814D100BF00BF2278920090
:1033A0002968895A494A114008460121C903014345
:1033B0008122D201114323789B002A68D15200BF99
:1033C00000BF2420005D01287ED16069C0196061C2
:1033D000E069C019E0612169206A884204D3266946
:1033E000206A801B20620DE0206A002804D13E463E
:1033F00000212420015505E0266A002020620021DA
:103400002420015500BF286803906078002846D129
:1034100000BF29680191296840310A8A0199511831
:1034200001912178C900891D01239B02019AD218BC
:10343000881800BF01888905890D01803E2E13D9A7
:1034400000BF71090091F106C90E002902D100994F
:10345000491E00910188009A92020123DB031A435E
:1034600092B21143018018E0002E05D1018801229B
:10347000D2031143018010E000BF71080091F107F1
:10348000C90F002902D00099491C00910188009AB7
:103490009206120C1143018000BF00BF13E0607858
:1034A000012810D128684030018A03980818039039
:1034B0002078C000801D01229202039989184018CB
:1034C00002900298068003E00AE000008F8F00005F
:1034D00000BFB3B2628961692868039004F02EFED0
:1034E00000BF227892002968895A094A114008468B
:1034F0001021484020214840890201438022114385
:1035000023789B002A68D15200BF002007B0F0BD8D
:10351000BF8F000002464807400F28235843134638
:10352000FF336933C018C0697047FFB581B00546E5
:103530000E461F460020009080203040802808D191
:103540007007400F28214843691844180120607013
:1035500009E07007400F282148432946FF316931AF
:103560004418002060707007400F2070039820619D
:10357000E770022F01D10020207100BF152040010B
:103580002818007A012802D1022005B0F0BD0120E0
:10359000152149016918087200BF2146286803F007
:1035A0004FFC00BF0020152149016918087200BFB7
:1035B0000098EAE7FFB581B005460E46174670074A
:1035C000400F282148432946FF316931441867617B
:1035D0000498A0610020E06160707007400F2070C7
:1035E0002146286804F06AF8002005B0F0BD70B5E7
:1035F00004460E467007400F6168884201D90120D9
:1036000070BD80203040802808D17007400F2821ED
:103610004843611845180120687007E0282070436E
:103620002146FF3169314518002068700120A870DB
:103630007007400F287000BF152040012018007A45
:10364000012801D10220DBE7012015214901611881
:10365000087200BF2946206804F002F800BF00206D
:10366000152149016118087200BF00BFC8E7FFB506
:1036700081B005460E461F467007400F282148437B
:103680006918441803986061A7610121242001553D
:1036900027620020E061012060707007400F2070F9
:1036A0002146286804F00AF8002005B0F0BD0000AB
:1036B00070B50446206804F015FD05460120C003DE
:1036C00028400121C903884203D1204601F0AEFA07
:1036D00070BD0120800228400121890288420FD15B
:1036E00020684030808872490840216840318880D5
:1036F000204600F08BF90021204600F0BCF9E7E7F6
:1037000001208003284001218903884208D12068D4
:103710004030808867490840216840318880D7E779
:1037200001204003284001214903884208D1206834
:103730004030808860490840216840318880C7E770
:103740000120000328400121090388422BD1206871
:10375000403000885949084021684031088020687D
:10376000403000885549091F0840216840310880D1
:103770001720400120180078012808D100201721C7
:1037800049016118087000212046FFF798FA204689
:1037900000F052F92068403080884949084021688B
:1037A0004031888094E70120C00228400121C902ED
:1037B00088421BD1206840300088082108432168D6
:1037C000403108802068403080883E4908402168A8
:1037D00040318880206840300088042108432168F7
:1037E00040310880204600F093F971E7802028409E
:1037F000802836D120684030808830497C390840A4
:103800002168403188801720400120180078002866
:1038100023D12068403000880421084321684031CA
:103820000880206840300088082108432168403122
:103830000880012017214901611808702068403074
:10384000808AF021084080080521C9016118486676
:1038500001212046FFF733FA02E0204600F058F934
:1038600036E70120400228400121490288420BD15D
:1038700020684030808814490840216840318880A1
:10388000204600F0EFF823E7FF2001302840FF2119
:103890000131884209D12068403080880749FC39CD
:1038A000084021684031888012E700BF10E700001F
:1038B000FFFB0000FFBF0000FFDF0000FBFF000078
:1038C000FFEF0000FFF70000FFFD000030B585B0FE
:1038D0000446002C02D1012005B030BD1520400166
:1038E0002018407A002806D1152149016118087274
:1038F000204600F067F8032015214901611848723D
:10390000206803F035FE00251CE0012228206843D2
:103910002146283140184270282068430D54002267
:10392000282068434018C27028206843401802616C
:10393000282068434018426128206843401882616B
:10394000681CC5B26068A842DFD800251CE00022D0
:10395000282068432146FF316931401842702820F1
:1039600068430D54282068434018C27028206843DB
:1039700040180261282068434018426128206843AB
:1039800040188261681CC5B26068A842DFD8142262
:10399000214610316846FCF755FC20460FC803F05D
:1039A000D9FD00212420015501201521490161186C
:1039B0004872E069012802D12046FFF766F900202D
:1039C0008AE7000038B504460E492068884217D1BE
:1039D00000BF0D48C0690121C90508430A49C861F3
:1039E0000846C0690121C9050840009000BF00BF1A
:1039F000002211461F20FFF73FF91F20FFF72EF985
:103A000038BD0000005C00400010024070B5044664
:103A10000125A068022801D0FEF798F90521C90107
:103A20006118086F294602F093FE0521C90161184B
:103A3000086F02F02BFE70BD10B50446A069002887
:103A400007D007480069062188430549086101F04D
:103A500033FE0521C9016118086F02F050FE10BD48
:103A600000ED00E010B504460521C9016118086F9A
:103A700002F056FE10BD70B504460D4600BF15207D
:103A800040012018007A012801D1022070BD0120D8
:103A9000152149016118087200BF242005552946E7
:103AA000206804F043FB00BF002015214901611884
:103AB000087200BF00BFE9E710B504460521C9013F
:103AC0006118086F2B210901611802F058FE10BD22
:103AD00010B5044600BF152040012018007A0128C7
:103AE00001D1022010BD0120152149016118087281
:103AF00000BF206804F0E2FA206803F021FD00BF57
:103B00000020152149016118087200BF00BFE9E7D4
:103B100010B504460521C9016118086F02F099FE2D
:103B2000A069002805D0034800690621084301491F
:103B3000086110BD00ED00E0F8B504460026002540
:103B4000012109042068084088427AD10027604892
:103B5000C0690903084000280DD100BF5C48C06956
:103B600008435B49C8610846C069090408400090E1
:103B700000BF00BF012757480068FF2101310840FE
:103B8000002816D153480068084352490860FEF7E0
:103B90002BFD064606E0FEF727FD801B642801D9B1
:103BA0000320F8BD4B480068FF2101310840002880
:103BB000F1D04748006A0321090208400546002D5C
:103BC0002DD060680840A84229D04148006A884347
:103BD00005463F48006A0121090408433C49086240
:103BE0000846006A012109048843394908620846E9
:103BF0000562E807C00F002811D0FEF7F5FC064665
:103C000007E0FEF7F1FC801B3349884201D903200D
:103C1000C7E72F48006A022108400028F1D02C484D
:103C2000006A032109028843616808432849086241
:103C3000012F05D10846C069090488432449C86199
:103C400000BF2078C007C00F002807D02048006BB5
:103C500080088000A16808431D490863022120688C
:103C60000840022808D11A48006B03210904884340
:103C7000E16808431649086320212068084020288D
:103C800007D11348006B102188432169084310496C
:103C900008630121490420680840884207D10C4884
:103CA000006B80218843A169084309490863012109
:103CB000890220680840884207D10548006B4021EE
:103CC00088436169084302490863002069E70000EE
:103CD00000100240007000408813000070B50446D8
:103CE0000D46002C01D1012070BD58480068C00766
:103CF000C00FA8420ED25548006840084000284333
:103D00005249086008460068C007C00FA84201D0A9
:103D10000120E9E7022120680840022814D104218B
:103D200020680840042807D1494840680721090253
:103D3000884340184649486045484068F021884318
:103D4000A1680843424948602078C007C00F002896
:103D500047D06068012808D13D4800680121490426
:103D60000840002821D10120BEE76068022808D160
:103D700037480068012149060840002815D1012074
:103D8000B2E76068032808D13148406B012149043B
:103D90000840002809D10120A6E72D48006802212B
:103DA0000840002801D101209EE72948406880088A
:103DB00080006168084326494860FEF715FC064606
:103DC00007E0FEF711FC801B2249884201D903203D
:103DD0008AE71F4840680C210840616889008842D2
:103DE000EFD11A480068C007C00FA8420ED9174883
:103DF00000684008400028431449086008460068ED
:103E0000C007C00FA84201D001206DE7042120683F
:103E10000840042808D10E48406807210902884359
:103E2000E16808430A49486000F01AF808494968FF
:103E3000F02211400909084A515CC840074908604E
:103E40000320FEF7C1FE00204EE7000000200240E4
:103E50000010024088130000F09500089C0000202C
:103E6000F8B50025002400270026002000902B48EC
:103E700045680C202840002849D0042804D0082890
:103E800005D00C2842D13EE02548009042E00F20AA
:103E900080042840800C23490E5C2048C06A00073B
:103EA000000F21490C5C0320C003284001210904B4
:103EB00088420AD12246002319481946FCF7FAF92C
:103EC000314604F059F907461BE00320C00328409F
:103ED0000321C90388420AD1224600231348194608
:103EE000FCF7E8F9314604F047F9074609E02246B5
:103EF00000230B481946FCF7DDF9314604F03CF984
:103F00000746009706E00948009003E000BF044818
:103F1000009000BF00BF0098F8BD000000100240F4
:103F200000127A00D0950008E0950008006CDC02D1
:103F3000FEB50446002C01D10120FEBD2078C0074B
:103F4000C00F002872D0FC4840680C2108400428AB
:103F50000CD0F94840680840082813D1F64840685A
:103F6000490308400121090488420BD1F248006846
:103F700001214904084000286BD06068002868D1FE
:103F80000120DAE700BF6068012807D1EA4800682D
:103F9000012109040843E849086031E0606800280D
:103FA0000ED1E5480068012109048843E249086010
:103FB00008460068012189048843DF4908601FE042
:103FC000606805280ED1DC48006801218904084397
:103FD000D949086008460068012109040843D64908
:103FE00008600DE0D4480068012109048843D249E3
:103FF000086008460068012189048843CE490860AA
:1040000000BF6068002812D0FEF7EEFA054606E011
:10401000FEF7EAFA401B642801D903208DE7C64861
:1040200000680121490408400028F1D011E0FEF7A2
:10403000DBFA054606E0FEF7D7FA401B642801D9F3
:1040400003207AE7BC4800680121490408400028A1
:10405000F1D1022120680840022862D1B6484068A8
:104060000C21084000280CD0B348406808400828BC
:104070001CD1B1484068490308400121C903884266
:1040800014D1AD48006802210840002804D0E0683F
:10409000012801D0012050E7A7480068F821884393
:1040A0002169C9000843A44908603AE0E068002893
:1040B00020D0A1480068012108439F490860FEF70D
:1040C00093FA054606E0FEF78FFA401B022801D955
:1040D000032032E798480068022108400028F2D007
:1040E00095480068F82188432169C900084392492E
:1040F000086016E090480068400840008E4908605B
:10410000FEF772FA054606E0FEF76EFA401B02283B
:1041100001D9032011E788480068022108400028DF
:10412000F2D1082120680840082831D1E069002830
:1041300017D08148406A012108437F494862FEF751
:1041400053FA054606E0FEF74FFA401B022801D954
:104150000320F2E67848406A022108400028F2D0A5
:1041600016E07548406A4008400073494862FEF70F
:104170003BFA054606E0FEF737FA401B022801D954
:104180000320DAE66C48406A022108400028F2D198
:10419000042120680840042872D10020019066485C
:1041A000C0698906084000280ED100BF6248C06976
:1041B00008436149C8610846C06909040840009085
:1041C00000BF00BF012001905C480068FF21013161
:1041D0000840002816D1594800680843574908602C
:1041E000FEF702FA054606E0FEF7FEF9401B6428DA
:1041F00001D90320A1E651480068FF2101310840A0
:104200000028F1D000BFA068012806D14A48006A02
:1042100001210843484908622AE0A06800280BD120
:104220004548006A4108490043480162006A042188
:104230008843414908621BE0A06805280CD13E482C
:10424000006A042108433C4908620846006A0121CB
:104250000843394908620BE03748006A40084000CB
:10426000354908620846006A0421884332490862D9
:1042700000BFA068002813D0FEF7B6F9054608E095
:104280002BE0FEF7B1F9401B2D49884201D90320EC
:1042900053E62948006A022108400028F1D011E0C5
:1042A000FEF7A2F9054607E0FEF79EF9411B2448F8
:1042B000814201D9032040E61F48006A02210840DC
:1042C0000028F1D10198012806D11B48C0690121BD
:1042D000090788431849C86100BF102120680840B9
:1042E00010285FD1606901282CD11348406B04214C
:1042F0000843114948630846406B012108430E49B1
:104300004863FEF771F9054606E0FEF76DF9401BBC
:10431000022801D9032010E60748406B022108401B
:104320000028F2D00448406BF8218843A169C900F5
:1043300008430149486335E0001002400070004026
:10434000881300006069401D00280FD18648406B2B
:1043500004218843844948630846406BF821884318
:10436000A169C9000843804948631BE07E48406B4F
:10437000042108437C4948630846406B40084000DC
:104380004863FEF731F9054606E0FEF72DF9401BBC
:10439000022801D90320D0E57348406B0221084070
:1043A0000028F2D1202120680840202852D16E48F0
:1043B00040680C2108400C280AD06B48406808402F
:1043C000082811D1684840684903084088420BD149
:1043D0006548406B01214904084000283AD0206A12
:1043E000012837D00120A8E5206A002819D05E48AE
:1043F000406B0121090408435B494863FEF7F4F868
:10440000054606E0FEF7F0F8401B022801D903201C
:1044100093E55548406B0121490408400028F1D03C
:1044200018E05148406B0121090488434E49486314
:10443000FEF7DAF8054606E0FEF7D6F8401B02283C
:1044400001D9032079E54848406B0121490408401F
:104450000028F1D1606A00284FD0434840680C2101
:104460000840082864D0606A022847D13E480068A6
:104470000121090688433C490860FEF7B5F8054666
:1044800006E0FEF7B1F8401B022801D9032054E5ED
:10449000354800680121490608400028F1D100BFD5
:1044A0003148C06A00090001216B08432E49C862E7
:1044B000A16AE06A08432C4949687B22D2039143F0
:1044C00008432949486000BF0846006801210906E1
:1044D000084325490860FEF787F8054606E0FEF721
:1044E00083F8401B022801D9032026E51E480068F6
:1044F0000121490608400028F1D033E01A4800683D
:1045000001210906884318490860FEF76DF8054641
:1045100006E0FEF769F8401B022801D903200CE5EC
:10452000114800680121490608400028F1D119E02E
:10453000606A012800D100E50B484668C76A03207D
:10454000C0033040A16A88420AD13907090F206BA5
:10455000814205D10F2080043040E16A884201D0B9
:104560000120EAE40020E8E40010024070B50446AF
:104570002546681E0949884201D901200CE0681EC1
:10458000074948610321081F03F032FE0020044957
:10459000886107200861002070BD0000FFFFFF0058
:1045A00000E000E000BFFEE70168896902221140D7
:1045B0004908002902D000210268916201688969D6
:1045C000C907C90F012251405140002904D1016897
:1045D000896911430268916170470000F7B584B0A2
:1045E00004460E460020039020688769002506983F
:1045F000029010203840102854D12168C8613DE055
:10460000701C00283AD0FDF7EFFF0299401AB04223
:1046100001D8002E32D1206840680121890308406A
:1046200001904220005D00902068806949000840A8
:10463000C00B00280ED04910019888420AD000987B
:10464000202807D020684068084321684860FDF7AB
:10465000CBFF02900AE0FDF7C7FF0299401A192824
:1046600004D9202005430120039006E020688069DA
:104670002021084040090028EDD000BF2068806953
:10468000202108404009002802D103980028B7D013
:104690000398002802D120202168C8610420054326
:1046A0000120039020688769FF2001303840FF21F6
:1046B0000131884206D10120054300022168C8610A
:1046C00001200390012080023840012189028842A4
:1046D00006D108200543C0012168C861012003906C
:1046E00001204002384001214902884206D10220BF
:1046F000054300022168C861012003900398002847
:1047000015D02046FFF750FF20684068094908404F
:1047100021684860606C2843606420214120015575
:1047200000214220015500BF4020015500BF0398E1
:1047300007B0F0BD00E800FEFFB581B004461546A5
:104740001E460A9F1B48F2B20023009020460299A1
:1047500000F032F8394620460B9A00F0B4F80028F1
:1047600002D0012005B0F0BD012E03D1E8B22168CE
:10477000886211E0FF200002284000122168886250
:10478000394620460B9A00F09EF8002801D00120FF
:10479000E8E7E8B2216888620B983B460022402196
:1047A0000090204600F026F8002801D00120D9E72B
:1047B0000020D7E700200080F8B5069C8D05AD0DE0
:1047C0001604FF273F043E4035431D4325436D003B
:1047D0006D08009505686E68650D0127BF023D40B4
:1047E000034F3D43AE43009D2E4305686E60F8BD08
:1047F000FF63FF03F8B504460D4617461E4623E047
:10480000701C002820D0FDF7EFFE0699401AB04238
:1048100001D8002E18D1206880692840A84201D113
:10482000012000E00020B8420ED1606C2021084336
:1048300060644120015500214220015500BF402005
:10484000015500BF0120F8BD206880692840A842BA
:1048500001D1012000E00020B842D1D00020F2E7D1
:1048600070B504460D46164624E0324629462046D9
:10487000FFF7B4FE002801D0012070BDFDF7B4FEA3
:10488000801BA84201D8002D14D120688069202106
:104890000840400900280DD1606C08436064412045
:1048A000015500214220015500BF4020015500BFA5
:1048B0000120E2E7206880692021084040090028A3
:1048C000D3D00020D9E770B504460D46164628E03F
:1048D000324629462046FFF781FE002801D00120FC
:1048E00070BD681C00281CD0FDF77EFE801BA8420E
:1048F00001D8002D15D120688069022108404008A8
:1049000000280ED1606C20210843606441200155CD
:1049100000214220015500BF4020015500BF012069
:10492000DEE7206880690221084040080028CFD0D7
:104930000020D5E730B50B46002100BF12E0040F80
:104940000A2C04D2040F30344D005C5503E0040FF0
:1049500037344D005C55000100254C00641C1D558A
:104960004C1CE1B29142EADB30BDF8B50546012DA1
:1049700017DA0026FF27002409E0204600F014F88B
:10498000002802D0701CC6B22746601CC4B2012C9D
:10499000F3DB012E03D1AF4201D10120F8BD00208D
:1049A000FCE70020FAE7000010B50146C8000B4BF9
:1049B00018580069CB00094C1B199B881840002827
:1049C00001D1002200E00122C800044BC018807908
:1049D000904201D1012010BD0020FCE7C8950008DD
:1049E00000B587B0142102A8FBF75EFD00BF4D485B
:1049F00040690121890508434A49486108464069E0
:104A0000012189050840019000BF00BF00BF454853
:104A100040694911084343494861084640690121FA
:104A200049040840019000BF00BF00BF3D484069F5
:104A3000490008433B49486108464069012189040F
:104A40000840019000BF00BF0022E7210920C006F6
:104A5000FDF7C3FD0122292189023348FDF7BDFD81
:104A6000002232493048FDF7B8FDE72002900120CE
:104A7000039000200490059002A90920C006FDF7CC
:104A8000A5FC1820029000200390049002A90920A0
:104A9000C006FDF79BFC03200290002003900490C9
:104AA00002A92148FDF792FC214802902120000430
:104AB00003900120049002A91B48FDF787FC2120E8
:104AC00080020290112003900120049000200590A4
:104AD00002A91548FDF77AFC1648029001200390C0
:104AE00000200490059002A90F48FDF76FFC0120FB
:104AF000400302900120039004900320059002A936
:104B00000948FDF763FC0120800302901120039007
:104B1000012004900320059002A90348FDF756FCEC
:104B200007B000BD00100240000400480848000023
:104B3000041000000808000010B51348134908606D
:104B4000134848600021114881600121C1600021A3
:104B5000016141618161C1610162FDF7BBFD002816
:104B600001D0FDF7F3F800210848FDF743FD0028C8
:104B700001D0FDF7EBF800210448FDF772FD002895
:104B800001D0FDF7E3F810BD00540040680200209A
:104B90000E09002010B500220F49104801F07FFBDC
:104BA000002801D0FDF7D2F80D490C4801F08DFE28
:104BB000002801D0FDF7CAF80A49084800F0ABFF09
:104BC000002801D0FDF7C2F8044801F065FF002875
:104BD00001D0FDF7BBF810BD280000200C03002019
:104BE000B00000208000002000BFFEE710B5FDF7F8
:104BF000D3FBFDF7B9FB0C48FDF71AFB0A48007B15
:104C0000BB280BDA022008490860BB20087308465D
:104C1000FDF71CFB002801D1FDF78AFBFDF798FB8F
:104C2000FDF77CFB10BD000030020020F0B587B01E
:104C300005469AE228684030808805900598070765
:104C40003F0F002F7ED1102105980840002836D153
:104C500000BF29680988FB4A114008460121C903A1
:104C600001432A68118000BF2C4628342868403050
:104C7000008A2178C9004018801C0122920229680C
:104C80008918405A8005800DE061E169606940182B
:104C9000606100212846FEF734F82420405D00289A
:104CA000C7D0A0690028C4D12420405D80210843DA
:104CB00029684031888100212420415555E22C4645
:104CC000FF346934286806880120C002304000287B
:104CD00028D028684030008A2178C9004018801DFB
:104CE0000122920229688918405A8005800DE061EE
:104CF000A08B83B2E288286803902B20000129183A
:104D0000039803F0F3F900BF29680988CE4A1140DF
:104D10000846802101432A68118000BF2846FEF71B
:104D2000CBFE22E20120C00330400028C6D000BFE5
:104D300029680988C44A11400846802101432A682D
:104D4000118000E08FE000BF28684030008A2178A1
:104D5000C9004018801D0122920229688918405A12
:104D60008005800DE061E069002812D060690028AC
:104D70000FD0A08B83B2E28861692868039003F0AA
:104D8000B5F9E16960694018606100212846FDF7C6
:104D9000C9FF286806880120C002304000288DD154
:104DA00003200003304003210903884286D000BF5E
:104DB00029680391296840310A8A0399511803919F
:104DC0000122920203998918881D00BF0188890574
:104DD000890D018021693E2915D900BF2169490942
:104DE0000291217CC906C90E002902D10299491EEF
:104DF00002910188029A92020123DB031A4392B2C4
:104E0000114301801BE02169002905D1018801229D
:104E1000D2031143018012E000BF216949080291C9
:104E2000217CC907C90F002902D00299491C0291AF
:104E30000188029A9206120C1143018000BF00BF44
:104E400000BF00BF29680988804A11400846012137
:104E5000090348404900484089000143802211432A
:104E60002A68118081E1B9002868465A0120C003F0
:104E70003040002871D000BFBA002968895A724AB0
:104E80001140084680210143BB002A68D15200BF6F
:104E9000282078432946FF3169314418207B0028B7
:104EA00019D128684030008A2178C9004018801D37
:104EB0000122920229688918405A8005800D0690C7
:104EC0000698002863D0E288616928680390069BF1
:104ED00003F00CF95BE0E078022806D13246214667
:104EE0002846FDF7ADFF069051E000BF00BF2278D5
:104EF00092002968895A534A80321140084601219C
:104F0000C9030143C022114323789B002A68D15270
:104F100000BF00BF217889002868405A0121890319
:104F2000084000281AD028684030008A2178C9003B
:104F30004018801C0122920229688918405A800575
:104F4000800D06900698002821D022896169286882
:104F50000390069B03F0CAF819E030E0286840305F
:104F6000008A2178C9004018801D01229202296818
:104F70008918405A8005800D06900698002806D0B2
:104F80006289616928680390069B03F0AFF8E169C4
:104F900006980818E0616169069808186061A069C0
:104FA000002803D021690698814204D92178284637
:104FB000FDF7B8FE03E02146286802F07FFB802061
:104FC000304000287AD028207843294628314418D8
:104FD00000BFBA002968895A1A4A114008460121BF
:104FE000C9030143BB002A68D15200BFE078012801
:104FF0007ED10020A061207B002876D04020304068
:10500000002839D000BF6078002821D100BF29686E
:105010000391296840310A8A039951180391217834
:10502000C900891C01239B02039AD218881800BF6B
:1050300001888905890D018001885A011143018089
:1050400000BF18E00F8F00008F0F00008FBF00001F
:10505000607801280FD100BF286829684031098A8B
:1050600008182178C900891C0122920282188B1825
:1050700000221A8000BF38E000BF286803906078E3
:1050800000281CD100BF29680191296840310A8A93
:105090000199511801912178C900891D01239B02B2
:1050A000019AD218881800BF01888905890D0180EE
:1050B00001885A011143018000BF15E055E0607876
:1050C000012811D128684030018A039808180390FC
:1050D0002078C000801D012292020399891840188F
:1050E000029000210298018000BF2178284600E04C
:1050F00002E0FDF706FE38E0FF20013030400028D6
:105100002ED128684030008A2178C9004018801CC0
:105110000122920229688918405A8005800D049066
:10512000A1690498814204D9A1690498081AA06170
:1051300001E00020A061A069002804D12178284660
:10514000FDF7DFFD11E06169049808186061E1690D
:1051500004980818E0612146286802F0AFFA04E0DC
:10516000324621462846FDF717FF286840308088E0
:105170000121C9030840002800D05BE507B0F0BD5D
:1051800030B587B00024002503F06AFB002834D036
:105190007D23DB0010221A49002003F077FB002852
:1051A00001D107B030BD7D23DB00182201A91020FA
:1051B00003F06CFB00280AD0162101A8FCF7DAFFE7
:1051C00004466846458BAC4201D00020E9E76846BA
:1051D000408B00280FD0182201A90A48FBF732F8AB
:1051E00016210848FCF7C6FF04460648C58AAC42AB
:1051F00003D00020D5E70020D3E70120D1E700004D
:1052000010020020C401002010B500247D23DB0023
:1052100014220749282003F039FB0548048A12218B
:10522000FCF7A8FFA04201D0002010BD0120FCE740
:10523000DC0100207047000010B50122120300219C
:10524000022000F0EBF96420FCF7AAFF0021022005
:1052500000F02EF9124908800846008811490840DC
:10526000002803D110A004F05BF802E015A004F0C0
:1052700057F807221F21022000F0D0F91022132135
:10528000022000F0CBF900221F21022000F0C6F915
:105290000121022000F00CF90149088010BD000036
:1052A00004000020FF8F000052544C383230314649
:1052B0002052657365742053756363656564210DC1
:1052C0000A00000052544C38323031462052657387
:1052D0006574204661696C6564210D0A0000000058
:1052E00010B50022012189022148FDF776F901203D
:1052F000FCF756FF012291021D48FDF76EF90022CE
:1053000001210920C006FDF768F9002220210920AB
:10531000C006FDF762F9002202210920C006FDF750
:105320005CF9002204210920C006FDF756F97D2012
:10533000C000FCF735FF012211460920C006FDF729
:105340004CF9012220210920C006FDF746F901226F
:1053500002210920C006FDF740F90122042109209D
:10536000C006FDF73AF9C820FCF71AFF10BD00008F
:10537000000400487047000000B587B0142102A85F
:10538000FBF792F800BF1A484069012189040843DD
:105390001749486108464069012189040840019085
:1053A00000BF00BF4811029011200390012004901B
:1053B0000320059002A90F48FDF708F801225103C8
:1053C0000C48FDF70AF901208003029001200390A8
:1053D000002004900320059002A90648FCF7F6FF80
:1053E0000022012189030348FDF7F7F807B000BD4B
:1053F000001002400004004870B50025002423E09E
:10540000002C01DD6806050E0022012189031048E9
:10541000FDF7E3F8FFF7AEFF012291030C48FDF71B
:10542000DCF8FFF7A7FF012149030948FDF7CCF895
:10543000002801D0012005430022012189030448EE
:10544000FDF7CBF8601CC4B2012CD9DB284670BD37
:105450000004004870B50025002423E0002C01DD85
:105460006806050E0022012189031048FDF7B5F8F2
:10547000FFF780FF012291030C48FDF7AEF80121F0
:1054800049030A48FDF7A0F8002801D00120054390
:10549000FFF770FF0022012189030448FDF79DF802
:1054A000601CC4B2082CD9DB284670BD000400483B
:1054B000F8B505460E466807000EF106C90E08430A
:1054C000074600F03BF8FF2000F07CF8FF2000F0DA
:1054D00079F8FF2000F076F8FF2000F073F8012043
:1054E00000F044F8022000F041F8002000F03EF8FF
:1054F000384600F067F800F00BF8FFF77DFFFFF784
:10550000A9FF04462402FFF7A5FF04432046F8BD87
:1055100000B585B014216846FAF7C6FF01204003A4
:105520000090002001900120029069460248FCF79B
:105530004DFF05B000BD00000004004800B585B077
:1055400014216846FAF7B0FF0120400300900120C3
:105550000190002002900320039069460248FCF766
:1055600035FF05B000BD00000004004870B50546D9
:10557000002422E00022012189031148FDF72DF8C3
:105580000220204128400121091B08410246012137
:1055900049030B48FDF721F8FFF7ECFE01229103C8
:1055A0000748FDF71AF8FFF7E5FE002201218903FD
:1055B0000348FDF712F8601CC4B2022CDADB70BDA0
:1055C0000004004870B50546002422E000220121B5
:1055D00089031148FDF701F8802020412840072168
:1055E000091B08410246012149030B48FCF7F5FF5E
:1055F000FFF7C0FE012291030748FCF7EEFFFFF71B
:10560000B9FE0022012189030348FCF7E6FF601C74
:10561000C4B2082CDADB70BD00040048F8B50546BA
:105620000E4614466807000EF106C90E08430746E9
:10563000FFF784FFFF20FFF7C5FFFF20FFF7C2FF42
:10564000FF20FFF7BFFFFF20FFF7BCFF0120FFF7A0
:105650008DFF0120FFF78AFF0020FFF787FF384604
:10566000FFF7B0FF0220FFF781FFFF210902214071
:105670000812FFF7A7FFE0B2FFF7A4FF01225103D2
:105680000148FCF7AAFFF8BD00040048704700007D
:1056900010B5FDF77DFA02F012FF06480068401CC5
:1056A000044908600A2803D30020086002F0FCFEC9
:1056B00010BD00002000002010B500F001F810BD62
:1056C00000B599B034210CA8FAF7EEFE002008903E
:1056D00009900A900B901C2101A8FAF7E5FE2320FF
:1056E0000C9001200D900F9014901020109002202B
:1056F0001590C1031691C1041791002118910CA8AF
:10570000FEF716FC002801D0FCF720FB07200890CC
:105710000220099000200A900B90012108A8FEF7B2
:10572000DDFA002801D0FCF711FB074801900020AA
:105730000590079001A8FEF7FFF9002801D0FCF7BB
:1057400005FB19B000BD00002000020070470000FA
:105750000120C04301218907086103480068401CFB
:1057600001490860704700002400002010B50024A3
:1057700017210020FFF79CFE04460120C0032040B3
:10578000C413204610BD10B5002412210020FFF7DD
:105790008FFE04460120C0032040C413204610BDE4
:1057A00010B5002417210020FFF782FE0446E020F8
:1057B00020404411204610BD10B500220121C9032C
:1057C0000548FCF70AFF0120FCF7EAFC0122D1039F
:1057D0000148FCF702FF10BD0004004810B5044664
:1057E0000B480078A04212D0002C06D00022802165
:1057F0000920C006FCF7F1FE05E001228021092006
:10580000C006FCF7EAFE02480470FFF7D5FF10BDA2
:105810001C00002010B504460B480078A04212D0AE
:10582000002C06D0002240210920C006FCF7D5FE3E
:1058300005E0012240210920C006FCF7CEFE024807
:105840000470FFF7B9FF10BD1B000020F8B5044637
:105850000D460520C0012018866B0520C0012018C8
:10586000076C0520C0012018806B00282AD0142066
:105870006843214614314018806800281CD0282233
:105880006A433B462833D218116914226A432346DF
:105890001433D2189068FAF709FE00290CD11420AD
:1058A0006843224614328018816000231A46294634
:1058B000204600F0DEFF03E00021852080008151BA
:1058C0000020F8BD0220FCE770B504460E46052016
:1058D000C0012018856B3146204600F02BFE832145
:1058E000890048510520C0012018806B00280DD088
:1058F0008121890048590521C9016118C96BCA680D
:105900008321890069189047002070BD0220FCE7C0
:1059100070B504460E4600258121204600F0F6FCB5
:105920000021E1620121204600F0F0FC0021FF206F
:105930006D3001518221204600F0E8FC00212164F5
:105940000520C0012018806B002810D00521C90156
:105950006118C96B486880470521C9016118886BC7
:1059600001F066FA00200521C90161188863284604
:1059700070BD000070B505460520C0012818846B75
:105980000520C0012818C06B002813D00120400258
:10599000005DFF280ED008490A5D491E085D0521FB
:1059A000C9016918C96B8B6821469847FF210120FE
:1059B00040020155002070BD0102000001460A208E
:1059C0000880014870470000A400002001464320E1
:1059D00008800148704700002C0100200146432048
:1059E0000880014870470000E8000020014643207D
:1059F000088001487047000070010020F8B5044697
:105A00000F460026207C002812D101235B020222CF
:105A10008121204600F00AFE0121E1624B020222B0
:105A2000204600F003FE0121FF206D30015110E0FF
:105A3000402302228121204600F0F8FD0121E1628D
:105A400040230222204600F0F1FD0121FF206D30AD
:105A50000151082303228221204600F0E7FD0121A5
:105A600021648720800001F0E5F90521C901611852
:105A700088630520C0012018806B002801D1012611
:105A800023E00520C0012018856B0521C90161189C
:105A9000C96B086880470021852080004151001DA6
:105AA0004151207C002808D1812080004259031FE9
:105AB0000121204600F0D2FD07E0812080004259FC
:105AC00040230121204600F0C9FD3046F8BD70B5E5
:105AD00004460520C0012018856B0520C001201850
:105AE000806B002815D0207C002808D18120800000
:105AF0004259031F0121204600F0B0FD07E081203C
:105B00008000425940230121204600F0A7FD0020DB
:105B100070BD0220FCE702460220002904D00523C4
:105B2000DB01D318D9630020704702460520C0016D
:105B30001018836B81208000C1500020704710B581
:105B400003460520C0011818846B4120C000015194
:105B5000212000010251002010BDFEB505460C4673
:105B60000520C0012818866B0021019100910027B3
:105B700020786021084000282FD020286DD1E088AF
:105B8000002820D020788021084000280ED0E2880C
:105B900060780521C9016918C96B8B68314698473F
:105BA000E2883146284600F000F915E061780120CE
:105BB00040028155A179401C8155E2883146284632
:105BC00000F0CFF808E060780521C9016918C96BB9
:105BD00000228B682146984745E06078002804D071
:105BE0000A2814D00B2830D123E00520C001281842
:105BF000007F032805D102226946284600F0D5F827
:105C000004E02146284600F0A0F8022723E0052002
:105C1000C0012818007F032805D1012201A92846C8
:105C200000F0C3F804E02146284600F08EF8022771
:105C300011E00520C0012818007F032804D0214668
:105C4000284600F082F8022705E02146284600F0A9
:105C50007CF8022700BF00BF05E02146284600F07F
:105C600074F8022700BF00BF3846FEBD70B5054678
:105C70000520C0012818846B0520C0012818806BFE
:105C8000002818D0852080000059002811D101215A
:105C9000852080000151001F01592963005B83B2F8
:105CA0004120C00002598121284600F0E2FD002079
:105CB00070BD0120FCE70220FAE770B504460D46EE
:105CC0000520C0012018406B2946426820469047B5
:105CD000002070BD70B504460D460520C001201897
:105CE000007F012804D0022803D003280ED101E050
:105CF00000BF00BF6888012807D100200521C90125
:105D000061184862204600F063F804E02946204606
:105D100000F01BF800BF00BF70BD70B506460C4612
:105D200015462B4622460021304600F097FC002005
:105D300070BD70B506460C4615462B46224600211E
:105D4000304600F096FD002070BD70B504460D464B
:105D50008021204600F059FD0021204600F055FD2D
:105D600070BD70B504460E46154603200521C901D5
:105D700061184861FF205D300551001D05512B461B
:105D800032460021204600F069FC002070BD10B5AD
:105D900004460520C1016118486100231A461946CE
:105DA000204600F05BFC002010BD70B504460E4696
:105DB000154602200521C90161184861E561256287
:105DC0002B4632460021204600F053FD002070BDD6
:105DD00010B5044604200521C9016118486100235B
:105DE0001A461946204600F044FD002010BD000070
:105DF00070B505460C46002D05D12246054906A082
:105E000000F00FFA04E02246024903A000F009FA6C
:105E1000004870BDD005002043444320436F6E66A8
:105E200069670000024612200880014870470000A0
:105E30004400002070B505460C46002D05D12246D1
:105E4000054906A000F0EDF904E02246024903A04E
:105E500000F0E7F9004870BDD0050020434443201E
:105E6000496E746572666163650000000246042035
:105E700008800148704700005800002070B50546B2
:105E80000C462246024903A000F0CBF9004870BD41
:105E9000D005002053544D6963726F656C6563745F
:105EA000726F6E696373000070B505460C46002D75
:105EB00005D12246054906A000F0B3F904E02246C8
:105EC000024903A000F0ADF9004870BDD0050020E4
:105ED00053544D3332205669727475616C20436F90
:105EE0006D506F727400000070B505460C461A20A4
:105EF0002080FCF727F9014870BD00005C000020FD
:105F000070B504460D46E888012804D0294620468D
:105F1000FFF71BFF20E00520C0012018007F0128AB
:105F200004D0022803D0032810D109E000BF0020CC
:105F3000A0600122214608312046FFF736FF0AE023
:105F40000122211D2046FFF730FF04E029462046AC
:105F5000FFF7FBFE00BF00BF70BDF8B504460E465C
:105F6000002000900027002570880012030002F036
:105F70001BF908F2050F28F2F2C9DCF2207C05219A
:105F8000C9016118096B0A68694690470746E9E04C
:105F9000207C00280AD10520C0012018406B816AAE
:105FA0006846884707460220787009E00520C0014E
:105FB0002018406BC16A68468847074602207870FF
:105FC000D0E0B078030002F0EFF806041C344C6413
:105FD0007C940520C0012018006B4068002809D07F
:105FE000207C0521C9016118096B4A686946904700
:105FF000074605E031462046FFF7A7FE681CC5B2FC
:106000007EE00520C0012018006B8068002809D0C0
:10601000207C0521C9016118096B8A68694690478F
:10602000074605E031462046FFF78FFE681CC5B2E3
:1060300066E00520C0012018006BC068002809D068
:10604000207C0521C9016118096BCA68694690471F
:10605000074605E031462046FFF777FE681CC5B2CB
:106060004EE00520C0012018006B0069002809D00F
:10607000207C0521C9016118096B0A6969469047AE
:10608000074605E031462046FFF75FFE681CC5B2B3
:1060900036E00520C0012018006B4069002809D0B7
:1060A000207C0521C9016118096B4A69694690473E
:1060B000074605E031462046FFF747FE681CC5B29B
:1060C0001EE00520C0012018006B8069002809D05F
:1060D000207C0521C9016118096B8A6969469047CE
:1060E000074605E031462046FFF72FFE681CC5B283
:1060F00006E031462046FFF728FE681CC5B200BF07
:1061000000BF2FE0207C002808D10520C001201806
:10611000406B416B68468847074605E0314620469C
:10612000FFF713FE681CC5B21CE0207C00280AD1D2
:106130000520C0012018406B016B68468847074660
:106140000720787005E031462046FFF7FEFD681C09
:10615000C5B207E0FFE731462046FFF7F6FD681CB1
:10616000C5B200BF00BF002D00D0F8BD6846008852
:10617000002812D0F08800280FD0F08869460988DE
:10618000884202DD6846008800E0F0880090694699
:106190000A8839462046FFF708FEF088002802D119
:1061A0002046FFF715FE00BFDFE70146002002E0B2
:1061B000421CD0B2491C0A78002AF9D1704770B548
:1061C00004460D460520C0012018007F012804D098
:1061D000022803D003281DD101E000BF00BFE888DA
:1061E000022804D029462046FFF7AFFD17E0012022
:1061F000E0600520C0012018406A002803D0022179
:10620000E0680843E060022221460C312046FFF797
:10621000CCFD04E029462046FFF797FD00BF00BFF4
:1062200070BDF8B504460D4617460026002C1ED05A
:106230002046FFF7BAFF4000801C38803A7830468D
:10624000711CCEB22A5403223146701CC6B26A5465
:106250000AE022783046711CCEB22A54641C002217
:106260003046711CCEB22A5420780028F1D1F8BDF6
:1062700001460020002906D0012906D0022906D0B7
:10628000032908D105E0002007E0022005E00120F5
:1062900003E0022001E0022000BF00BF704770B59C
:1062A00004460D461646002C01D1022070BD052083
:1062B000C0012018406B002804D000200521C9012E
:1062C00061184863002D03D00520C0012018056324
:1062D00001200521C901611808772670204600F0C9
:1062E00035F90020E2E7F8B504460D460026002700
:1062F0000521C9016118086C2946FCF75EFD0646B8
:106300003046FFF7B5FF07463846F8BDF8B50446F6
:106310000D46002600270521C9016118086C294691
:10632000FCF712FD06463046FFF7A2FF0746384647
:10633000F8BDF8B504460E461746002E7AD125461C
:1063400014350520C00120184069022852D129695E
:10635000E868884210D92969E868401AE860A88985
:1063600082B239462046FFF7E4FC00231A4619465C
:10637000204600F073F94DE02969A868FAF796F80D
:1063800000291BD12969A868884217D30521C901B2
:106390006118A8688969884210D2002211462046F7
:1063A000FFF7C7FC00200521C9016118886100239F
:1063B0001A461946204600F051F92BE00520C0018D
:1063C0002018406BC06800280CD00520C0012018A0
:1063D000007F032806D10520C0012018406BC1684A
:1063E000204688478021204600F00FFA2046FFF71C
:1063F000CEFC0FE00520C00120184069042805D01C
:106400000520C00120184069002803D180212046C2
:1064100000F0FBF91520400120180078012821D157
:10642000204600F05DFA002015214901611808702E
:1064300018E0FFE70520C0012018406B40690028E4
:106440000ED00520C0012018007F032808D10520A8
:10645000C0012018406B314642692046904701E058
:106460000220F8BD0020FCE7F8B504460E461746AA
:10647000002E45D12546FF3555350520C001201891
:10648000406903282CD12969E868884210D9296914
:10649000E868401AE8602969E868884201D2E8683B
:1064A00000E0286982B239462046FFF736FC3FE01B
:1064B0000520C0012018406B006900280CD0052081
:1064C000C0012018007F032806D10520C001201834
:1064D000406B0169204688472046FFF779FC27E09A
:1064E0000520C00120184069052821D10020052180
:1064F000C901611848610021204600F086F917E0C3
:106500000520C0012018406B806900280ED00520AE
:10651000C0012018007F032808D10520C0012018E1
:10652000406B314682692046904701E00220F8BD69
:106530000020FCE770B504460D460521C90161182D
:10654000086C2946FCF7E6FF70BD000010B5044654
:106550002548046725480521C901611808642448B5
:1065600022490860082048600221204881600161BA
:1065700000218161C1610162FDF7A8F9002801D005
:10658000FBF7E4FB0521C901611818230022086C00
:106590001146FCF795FB0521C9016118582300221B
:1065A000086C8021FCF78CFB0521C9016118C02310
:1065B0000022086C8121FCF783FB0521C9016118C9
:1065C000FF2311330022086C0121FCF779FB052120
:1065D000C9016118FF2301330022086C8221FCF7F6
:1065E0006FFB002010BD000050120020D00F0020D3
:1065F000005C004010B502460520C0011018036C75
:1066000080200840802807D14806400E2824604397
:106610001C190019807810BD4806400E28246043DC
:106620001C46FF34693400198078F4E7FEB504464F
:106630000F4615461E460020019000900521C90115
:1066400061182B463246086C3946FCF76EFF019004
:106650000198FFF70DFE00900098FEBDFEB50446C0
:106660000D4616461F460020019000900521C901E5
:1066700061183B463246086C2946FCF79BFF0190A7
:106680000198FFF7F5FD00900098FEBD10B5044697
:106690004023002211462046FFF7C8FF0121FF20BA
:1066A000593001514021FF20653001514023002223
:1066B00080212046FFF7BAFF0121A16140216162DC
:1066C00001200521C9016118087700200521C901B1
:1066D0006118486160600521C901611848620520A0
:1066E000C0012018806B002807D021790520C00147
:1066F0002018406B426820469047002010BD01469C
:106700000520C0010818007F042807D10520C0011A
:106710000818407F0522D2018A18107700207047A0
:1067200010B504460520C0012018007F03280DD1B4
:106730000520C0012018406BC069002806D0052044
:10674000C0012018406BC16920468847002010BD59
:106750000246117400207047F8B504460D46002625
:1067600000270521C9016118086C2946FDF783F946
:1067700006463046FFF77CFD07463846F8BD70B543
:1067800004460D4629465520C000201800F089F81F
:1067900001200521C901611848615520C000201859
:1067A000C0880521C90161188861152040012018A1
:1067B000007AC006C00E002804D0012809D00228A3
:1067C00015D10DE05520C0002118204600F06BF9CE
:1067D00018E05520C0002118204600F0E3FA11E02F
:1067E0005520C0002118204600F0B1F90AE015201C
:1067F00040012018007A802210400146204600F017
:1068000004F800BF00BF002070BDF8B504460D4677
:10681000002600270521C9016118086C2946FCF7EC
:10682000E6FE06463046FFF723FD07463846F8BD2C
:1068300070B50446002500260521C9016118086CC1
:10684000FDF746F905462846FFF712FD0646304695
:1068500070BD01460520C0010818007F0522D20145
:106860008A18507704200522D2018A181077002058
:106870007047FEB504460D4616461F46002001909F
:1068800000900521C90161183B463246086C294633
:10689000FCF7EDFE01900198FFF7EAFC00900098EC
:1068A000FEBD0A7802704A7842708B78CA7812026C
:1068B0009A1842800B794A7912029A1882808B7951
:1068C000CA7912029A18C280704702460020002935
:1068D00004D00523DB01D318596300E00220704780
:1068E00001460020704770B504460D46A888002870
:1068F0002CD1E888002829D16888802826D2A87859
:106900004606760E0520C0012018007F032804D11A
:1069100029462046FFF719FA1CE00520C00120187F
:10692000867731462046FFF717FF2046FFF750FADB
:10693000002E05D002200521C9016118087709E061
:1069400001200521C9016118087703E02946204686
:10695000FFF7FBF970BD70B504460D460226052011
:10696000C0012018406B00280AD00520C001201863
:10697000406B2946026820469047002800D1002637
:10698000304670BD70B504460D46A8783A49087087
:1069900008460078012804DD29462046FFF7D5F98E
:1069A00068E00520C0012018007F022802D00328DB
:1069B00055D11FE030480078002817D02E480078C5
:1069C000606003200521C901611808772A48017811
:1069D0002046FFF7C0FF022804D129462046FFF7D2
:1069E000B4F970BD2046FFF7F3F902E02046FFF747
:1069F000EFF93EE020480078002810D10220052160
:106A0000C901611808771C48007860601A4801784D
:106A10002046FFF752F92046FFF7DAF91EE0164943
:106A200009786068884216D021792046FFF745F939
:106A3000114800786060104801782046FFF78BFF0E
:106A4000022804D129462046FFF77FF9C9E72046EE
:106A5000FFF7BEF902E02046FFF7BAF909E0294640
:106A60002046FFF772F9044801782046FFF725F920
:106A700000BF00BF00BFB4E7A000002070B505460E
:106A80000C466088012806D10521C90169184862B1
:106A90002846FFF79DF970BD10B504462046FFF764
:106AA000C7FE002010BD70B505460C4600262078B4
:106AB0006021084000280ED0202802D040283ED176
:106AC00000E000BF0520C0012818406B2146826805
:106AD0002846904738E06078030001F065FB0A1A09
:106AE00024291F290B062915102921462846FFF7BE
:106AF00034FA22E021462846FFF7F5FE1DE0214644
:106B00002846FFF73FFF18E021462846FFF7F8F92F
:106B100013E021462846FFF752FB0EE021462846A7
:106B2000FFF7ACFF09E021462846FFF7D3F804E061
:106B300021462846FFF709F900BF00BF04E02146BF
:106B40002846FFF702F900BF00BF304670BDF8B518
:106B500005460E46002000903479307860210840C8
:106B600000280ED0202802D0402870D100E000BFBD
:106B70000520C0012818406B31468268284690479E
:106B80000DE130786021084020280AD10520C0019D
:106B90002818406B3146826828469047009000983C
:106BA000F8BD7078002869D0012835D0032877D146
:106BB0000520C0012818007F022802D0032824D114
:106BC00011E0002C0AD0802C08D021462846FFF77F
:106BD0001CFE80212846FFF718FE03E031462846B8
:106BE000FFF7B3F816E0708800280AD1002C08D00F
:106BF000802C06D0F088002803D121462846FFF7D4
:106C000004FE2846FFF7E4F804E031462846FFF783
:106C10009CF800BF00BFBBE00520C0012818007F22
:106C2000022802D0032822D112E0002C0AD0802CA6
:106C300008D021462846FFF7E8FD80212846FFF7C7
:106C4000E4FD03E031462846FFF77FF814E0A1E0B9
:106C5000708800280AD16006400E002803D0214623
:106C60002846FFF740FB2846FFF7B2F804E031461C
:106C70002846FFF76AF800BF00BF89E00520C00181
:106C80002818007F022802D0032875D125E0002CA7
:106C900007D0802C05D031462846FFF756F870E023
:106CA00071E080202040802806D16006400E14212B
:106CB00048436918401807E06006400E1421484315
:106CC0002946FF315531401807460020386002221E
:106CD00039462846FFF769F853E080202040802895
:106CE0000DD12007000F142148436918401840684F
:106CF000002814D131462846FFF727F841E0200745
:106D0000000F142148432946FF315531401840688F
:106D1000002804D131462846FFF717F831E08020DB
:106D20002040802806D16006400E1421484369188F
:106D3000401807E06006400E142148432946FF3101
:106D4000553140180746002C01D0802C02D100207C
:106D500038600AE021462846FFF74CFC002802D0A4
:106D60000120386001E000203860022239462846C0
:106D7000FFF71BF805E0FFE731462846FEF7E5FF81
:106D800000BF00BF04E031462846FEF7DEFF00BF2B
:106D900000BF04E031462846FEF7D7FF00BF00BF22
:106DA0000098FDE670B505460C4600262078602167
:106DB0000840002806D0202802D0402830D100E02A
:106DC00000BF00BF0520C0012818007F012804D0A3
:106DD000022803D003281CD101E000BF00BF2079A6
:106DE000012811DC0520C0012818406B214682686B
:106DF000284690470646E088002809D1002E07D192
:106E00002846FEF7E5FF03E021462846FEF79DFFF2
:106E100004E021462846FEF798FF00BF00BF04E0CB
:106E200021462846FEF791FF00BF00BF002070BD3D
:106E3000704700000146014870470000C41200205E
:106E4000FCB502460020019008788000105AFE4CE4
:106E500020400346C878002806D001280ED002281A
:106E600006D003280ED105E00120400203430CE0C8
:106E700000BF0AE003204002034306E00120800235
:106E8000034302E00120019000BF00BF1846EF4C11
:106E900020430C78A400105300BF0C78A400145BAE
:106EA000EB4D2C400D782C4320460124E403044391
:106EB00080252C430D78AD00545300BF087B00287B
:106EC0007ED1487800284ED000BF10465025AD5ADC
:106ED00028180D78ED000126B6028619AC19CD8868
:106EE0006D106D00258000BF00BF0C78A400105B02
:106EF00040240440002C0FD000BF0D78AD00555B3E
:106F0000D34E35402C460125ED032543C02635439D
:106F10000E78B600955300BF00BFC878012811D085
:106F200000BF0C78A400145BC94D30352C402046BE
:106F300020246040A402044380252C430D78AD003A
:106F40005453C5E100BF0C78A400145BC04D30352C
:106F50002C4020460124E403044380252C430D7873
:106F6000AD005453B4E100BF10465025AD5A281867
:106F70000D78ED002D1D0126B6028619AC19CD88BD
:106F80006D106D00258000BF00BF00925024A45AF0
:106F9000009AA41800940C78E400A41D0126B602FF
:106FA000009DAD196419204600BF0588AD05AD0DE3
:106FB00005800D693E2D13D900BF0D696C0900E0F5
:106FC0006CE00D7CED06ED0E002D00D1641E0588F1
:106FD000A6020127FF033E43B6B23543058017E002
:106FE0000D69002D05D105880126F603354305807E
:106FF0000EE000BF0D696C080D7CED07ED0F002D54
:1070000000D0641C0588A606360C3543058000BFF9
:1070100000BF00BF00BF0C78A400105B0124A403D4
:107020000440002C10D000BF0D78AD00555B884E99
:1070300035402C460125ED0325438126F6013543D5
:107040000E78B600955300BF00BF0878002813D112
:1070500000BF0C78A400145B7E4D2C402046012418
:107060002403604064006040A400044380252C4356
:107070000D78AD0054532BE100BF0C78A400145BD5
:10708000744D2C402046012464036040A400044356
:1070900080252C430D78AD00545319E1C87802289F
:1070A00010D100BF0C78A400145B694D2C40204621
:1070B0000124E4030443FF2581352C430D78AD0002
:1070C00054530FE000BF0C78A400145B624D2C40B9
:1070D00020460124E403044380252C430D78AD00B1
:1070E000545300BF00BF00BF00BF10465025AD5A2B
:1070F00028180D78ED000126B6028619AC190D8905
:107100006D106D00258000BF00BF00BF00BF10469E
:107110005025AD5A28180D78ED002D1D0126B60218
:107120008619AC194D896D106D00258000BF00BF18
:1071300000BF4878002858D100BF0C78A400105B2D
:107140000124A4030440002C10D000BF0D78AD0032
:10715000555B3F4E35402C460125ED0325438126E6
:10716000F60135430E78B600955300BF00BF00BF4F
:107170000C78A400105B40240440002C0FD000BF0A
:107180000D78AD00555B324E35402C460125ED03A0
:107190002543C02635430E78B600955300BF00BF87
:1071A00000BF0C78A400145B2A4D2C40204601241B
:1071B0002403604064006040A400044380252C4305
:1071C0000D78AD00545300BF00BF0C78A400145BD1
:1071D0001F4D30352C4020460124E4030443802514
:1071E0002C430D78AD00545372E000BF0C78A4001E
:1071F000105B0124A4030440002C10D000BF0D78C4
:10720000AD00555B124E35402C460125ED0325435C
:107210008126F60135430E78B600955300BF00BFB6
:1072200000BF08788000145A4020204000281AD05F
:1072300000BF0D78AD00555B054E35402846012551
:10724000ED030543C02609E08F890000808000001F
:107250008F8F00008FBF00008F8E000035430E78A7
:10726000B600955300BF00BFC878012810D000BFFA
:107270000C78A400145B174D2C402046202460405D
:10728000A402044380252C430D78AD0054530FE035
:1072900000BF0C78A400145B0E4D2C402046012446
:1072A000E403044380252C430D78AD00545300BF04
:1072B00000BF0C78A400145B074D2C40204601242D
:1072C000E403044380252C430D78AD00545300BFE4
:1072D0000198FCBDBF8F00008FBF000030B5024693
:1072E000087B002857D14878002829D000BF0B78A8
:1072F0009B00D05A40230340002B0FD000BF0C78D6
:10730000A400145B8C4D2C4023460124E4031C4351
:10731000C0252C430D78AD00545300BF00BF00BF03
:107320000B789B00D35A844C3034234018460123F9
:10733000DB030343802423430C78A4001353F8E0B9
:1073400000BF0B789B00D05A01239B030340002B06
:1073500010D000BF0C78A400145B774D2C4023465E
:107360000124E4031C438125ED012C430D78AD007D
:10737000545300BF00BF00BF0B789B00D35A6F4C23
:10738000234018460123DB030343802423430C7866
:10739000A4001353CDE04878002864D100BF0B78D7
:1073A0009B00D05A01239B030340002B10D000BF49
:1073B0000C78A400145B604D2C4023460124E403A8
:1073C0001C438125ED012C430D78AD00545300BFC3
:1073D00000BF00BF0B789B00D05A40230340002B16
:1073E0000FD000BF0C78A400145B534D2C402346F3
:1073F0000124E4031C43C0252C430D78AD005453F5
:1074000000BF00BF00BF0B789B00D35A4A4C2340FB
:1074100018460123DB030343C02423430C78A40054
:10742000135300BF00BF0B789B00D35A434C23403B
:1074300018460123DB030343802423430C78A40074
:10744000135300BF00BF0B789B00D35A3A4C303423
:10745000234018460123DB030343802423430C7895
:10746000A400135365E000BF0B789B00D05A0123A2
:107470009B030340002B10D000BF0C78A400145BCA
:107480002D4D2C4023460124E4031C438125ED01AE
:107490002C430D78AD00545300BF00BF00BF0B78E4
:1074A0009B00D05A40230340002B0FD000BF0C7824
:1074B000A400145B204D2C4023460124E4031C430C
:1074C000C0252C430D78AD00545300BF00BF00BF52
:1074D0000B789B00D35A184C234018460123DB033A
:1074E00003438124E40123430C78A400135300BF19
:1074F00000BF0B789B00D35A0F4C30342340184602
:107500000123DB030343802423430C78A40013539B
:1075100000BF00BF0B789B00D35A084C234018468D
:107520000123DB030343802423430C78A40013537B
:1075300000BF002030BD00008F8F00008FBF000013
:1075400001465820405A0122D2031043582250527B
:107550000020704710B5044601214020015300214E
:1075600001534420015350200153002010BD00005E
:107570000146044A4020405A90434023585200207C
:107580007047000080BF000030B50246087B00282D
:107590005FD1487800282DD000BF0B789B00D05ACF
:1075A00040230340002B0FD000BF0C78A400145BD5
:1075B000294D2C4023460124E4031C43C0252C43C1
:1075C0000D78AD00545300BF00BFC878012840D0EB
:1075D00000BF0B789B00D35A1F4C30342340184611
:1075E000202358409B020343802423430C78A400AB
:1075F00013532EE000BF0B789B00D05A01239B034E
:107600000340002B10D000BF0C78A400145B124D77
:107610002C4023460124E4031C438125ED012C4327
:107620000D78AD00545300BF00BF00BF0B789B0026
:10763000D35A0A4C2340184601231B0358405B00D1
:1076400058409B000343802423430C78A400135329
:1076500000BF002030BD00008F8F00008FBF0000F2
:1076600010B502464878002810D000BF0B789B0068
:10767000D35A104C2340184610235840DB020343D2
:10768000802423430C78A400135311E000BF0B782F
:107690009B00D35A084C2340184601231B03584033
:1076A000DB000343802423430C78A400135300BF62
:1076B000002010BDBF8F00008FBF0000F0B585B067
:1076C00006460C466078012873D12169A06988427A
:1076D00001D9256900E0A569207B002813D1ABB250
:1076E000E2883046616900F029FD00BF3046502233
:1076F000925B10182278D200921C01239B02C318BF
:10770000D1180D80AEE2E07802287DD12169206A8F
:1077100088427AD900BF21788900715AFE4A114007
:1077200008460121C9030143FF2281321143227817
:107730009200B15200BF206A401B20622078800076
:10774000305A4021084000287ED000BF0296607861
:1077500000283ED100BF00965021895B009E891908
:1077600000912178C900891D01239B02009AD2183B
:107770008918084600BF02889205920D02803E2DAE
:107780000FD900BF6909EA06D20E002A00D1491EAE
:1077900002888B020127FF033B439BB21A430280FE
:1077A00015E0002D06D102880123DB031A43028075
:1077B0000DE06AE200BF6908EA07D20F002A00D094
:1077C000491C02888B061B0C1A43028000BF00BFB5
:1077D00012E0607801280FD15020815B02980818D0
:1077E00002902078C000801D01229202029989181F
:1077F000401801900198058000BF60890490ABB2E9
:1078000061693046049A01E061E138E100F096FCDC
:107810006069401960612169206A884203D9206A41
:10782000401B206202E0256A0020206200BF6078D1
:1078300000283FD100BF02965021895B029E891922
:1078400002912178C90000E04FE0891C01239B02CE
:10785000029AD2188918084600BF02889205920D34
:1078600002803E2D0FD900BF6909EA06D20E002A18
:1078700000D1491E02888B020127FF033B439BB2C4
:107880001A43028014E0002D05D102880123DB0396
:107890001A4302800CE000BF6908EA07D20F002AF1
:1078A00000D0491C02888B061B0C1A43028000BFC3
:1078B00000BF10E0607801280DD100BF3046502293
:1078C000925B10182278D200921C01239B02C318ED
:1078D000D1180D8000BF00BF20890490ABB2616950
:1078E0003046049A00F02AFCBCE100BF6078002812
:1078F0003DD100BF02965021895B029E89190291F9
:107900002178C900891C01239B02029AD218891888
:10791000084600BF02889205920D02803E2D0FD9C5
:1079200000BF6909EA06D20E002A00D1491E02886A
:107930008B020127FF033B439BB21A43028014E0F2
:10794000002D05D102880123DB031A4302800CE0DD
:1079500000BF6908EA07D20F002A00D0491C02883C
:107960008B061B0C1A43028000BF00BF10E060783A
:1079700001280DD100BF30465022925B10182278AA
:10798000D200921C01239B02C318D1180D8000BFA6
:1079900000BF20890490ABB261693046049A00F0C0
:1079A000CDFB6069401960612169206A884203D972
:1079B000206A401B206202E0256A0020206200BF8E
:1079C0000296607800283DD100BF00965021895B67
:1079D000009E891900912178C900891D01239B020D
:1079E000009AD2188918084600BF02889205920DA5
:1079F00002803E2D0FD900BF6909EA06D20E002A87
:107A000000D1491E02888B020127FF033B439BB232
:107A10001A43028014E0002D05D102880123DB0304
:107A20001A4302800CE000BF6908EA07D20F002A5F
:107A300000D0491C02888B061B0C1A43028000BF31
:107A400000BF12E0607801280FD15020815B0298BE
:107A5000081802902078C000801D0122920202992D
:107A60008918401801900198058000BF6089049032
:107A7000ABB261693046049A00F060FBF2E0256A1F
:107A800000BF21788900715A244A1140084601211B
:107A9000C90301438022114322789200B15200BFF2
:107AA00000BF30465022925B10182278D200921C00
:107AB00001239B02C318D1180D8000BF20890490B8
:107AC000ABB261693046049A00F038FBCAE0206A24
:107AD000401B206220788000305A40210840002856
:107AE00064D000BF02966078002842D100BF0096A3
:107AF0005021895B009E891900912178C900891D58
:107B000001239B02009AD2188918084600BF0288F8
:107B10009205920D028003E08F8F00008F8E00008F
:107B20003E2D0FD900BF6909EA06D20E002A00D106
:107B3000491E02888B020127FF033B439BB21A4375
:107B4000028014E0002D05D102880123DB031A43D3
:107B500002800CE000BF6908EA07D20F002A00D0BB
:107B6000491C02888B061B0C1A43028000BF00BF11
:107B700012E0607801280FD15020815B029808182C
:107B800002902078C000801D01229202029989187B
:107B9000401801900198058000BF60890490ABB245
:107BA00061693046049A00F0C9FA5BE000BF607872
:107BB00000283DD100BF02965021895B029E8919A1
:107BC00002912178C900891C01239B02029AD218D4
:107BD0008918084600BF02889205920D02803E2D4A
:107BE0000FD900BF6909EA06D20E002A00D1491E4A
:107BF00002888B020127FF033B439BB21A4302809A
:107C000014E0002D05D102880123DB031A43028012
:107C10000CE000BF6908EA07D20F002A00D0491C17
:107C200002888B061B0C1A43028000BF00BF10E0C5
:107C3000607801280DD100BF30465022925B1018A9
:107C40002278D200921C01239B02C318D1180D8008
:107C500000BF00BF20890490ABB261693046049A2E
:107C600000F06CFA00BF21788900715AFA4A11407D
:107C700008461021484020214840890201438022C3
:107C8000114322789200B15214E2207B002849D19E
:107C90002169A069884204D92569A069401BA061B7
:107CA00002E0A5690020A06100BF02965021895B17
:107CB000029E891902912178C900891D01239B0226
:107CC000029AD2188918084600BF02889205920DC0
:107CD00002803E2D0FD900BF6909EA06D20E002AA4
:107CE00000D1491E02888B020127FF033B439BB250
:107CF0001A43028014E0002D05D102880123DB0322
:107D00001A4302800CE000BF6908EA07D20F002A7C
:107D100000D0491C02888B061B0C1A43028000BF4E
:107D200000BFB3E1E07802287ED100BF00BF6078D9
:107D3000002843D100BF02965021895B029E891919
:107D400002912178C900891C01239B02029AD21852
:107D50008918084600BF02889205920D02802269A8
:107D60003E2A11D900BF22695109227CD206D20EC7
:107D7000002A00D1491E02888B020127FF033B43E2
:107D80009BB21A43028017E02269002A05D10288BB
:107D90000123DB031A4302800EE000BF2269510871
:107DA000227CD207D20F002A00D0491C02888B0601
:107DB0001B0C1A43028000BF00BF11E0607801284D
:107DC0000ED100BF30465022925B10182278D200AC
:107DD000921C01239B02C318D118228A0A8000BF7B
:107DE00000BF00BF02966078002845D100BF009612
:107DF0005021895B009E891900912178C900891D55
:107E000001239B02009AD2188918084600BF0288F5
:107E10009205920D028022693E2A13D900BF226981
:107E20005109227CD20600E06DE0D20E002A00D17A
:107E3000491E02888B020127FF033B439BB21A4372
:107E4000028017E02269002A05D102880123DB03A2
:107E50001A4302800EE000BF22695108227CD2073B
:107E6000D20F002A00D0491C02888B061B0C1A4333
:107E7000028000BF00BF14E06078012811D15020BB
:107E8000815B0298081802902078C000801D0122B2
:107E900092020299891840180190208A81B20198B3
:107EA000018000BF00BFE06900282BD0207880004F
:107EB000305A03900121890303980840002804D018
:107EC00040210398084000280AD101218903039822
:107ED0000840002816D14021039808400028F9D115
:107EE00000BF00BF21788900715A5B4A303A1140C7
:107EF00008460121C9030143C022114322789200A0
:107F0000B15200BFC2E0E07801287DD12169A069AB
:107F1000884204D92569A069401BA06102E0A569D7
:107F20000020A06100BF00BF607800283DD100BFE5
:107F300002965021895B029E891902912178C9001D
:107F4000891C01239B02029AD2188918084600BF97
:107F500002889205920D02803E2D0FD900BF69095B
:107F6000EA06D20E002A00D1491E02888B020127A0
:107F7000FF033B439BB21A43028014E0002D05D15E
:107F800002880123DB031A4302800CE000BF69086A
:107F9000EA07D20F002A00D0491C02888B061B0C6E
:107FA0001A43028000BF00BF10E0607801280DD1A5
:107FB00000BF30465022925B10182278D200921CEB
:107FC00001239B02C318D1180D8000BF00BF00BF62
:107FD00002966078002841D100BF00965021895B4D
:107FE000009E891900912178C900891D01239B02F7
:107FF000009AD2188918084600BF02889205920D8F
:1080000002803E2D11D900E03DE000BF6909EA067B
:10801000D20E002A00D1491E02888B020127FF03DD
:108020003B439BB21A43028014E0002D05D1028825
:108030000123DB031A4302800CE000BF6908EA0752
:10804000D20F002A00D0491C02888B061B0C1A4351
:10805000028000BF00BF14E0BF8F000060780128DD
:108060000FD15020815B0298081802902078C00040
:10807000801D0122920202998918401801900198EE
:10808000058000BF02E0012005B0F0BD00BF2178EF
:108090008900715A084A11400846012109034840E5
:1080A0004900484089000143802211432278920010
:1080B000B15200BF0020E7E78FBF00000146002358
:1080C00044204352024A40204252002070470000A0
:1080D00080BF000010B50248FBF7EAFA10BD0000AF
:1080E000D00F002001464422505A7047FFB582B09D
:1080F00004465E080196009403980126B602009C8F
:10810000A6199519019F07E02988AD1C0170401C34
:108110000E0A0670401C7F1E002FF5D1DE07F60FF9
:10812000002E01D02988017006B0F0BD024600295A
:1081300002D180234C20835200207047FFB582B0CB
:1081400004460F46059E761C760801960094384634
:108150000126B602009CA6199519019B08E001783A
:108160004678360231432980AD1C401C401C5B1E02
:10817000002BF4D106B0F0BDF8B582B28BB2040C7E
:108180000D0C10465843002126465E43370C36043A
:108190008019794116466E43370C360480197941AF
:1081A00026466E438919F8BD30B47446641E25789E
:1081B000641CAB4204D3635D5B00E31830BC18471A
:1081C0001D46F8E74900CA020243100000D004200F
:1081D0004A0D01D001221043044A490D914201D1B8
:1081E00002210843012800D105207047FF07000045
:1081F00010B5002819DB1A4A03231B02D218830882
:108200009B00D2588307DC0EFF23A3409A438B07C1
:108210001B0E8407E40EA3401A43114B03242402CF
:108220001B198408A4001A5118E00E4A03071B0FFB
:10823000083B9B089B00D2588307DC0EFF23A3401A
:108240009A438B071B0E8407E40EA3401A43054B89
:108250000407240F083CA408A4001A5110BD000014
:1082600000E100E01CED00E030380A2801D20120D6
:10827000704700207047000070B50546280124496A
:1082800044182846FCF771FB002832D0A07A002859
:1082900007D10120A07269006918491CC8B200F01A
:1082A00019F92089002832DDE088218988420DDA19
:1082B000E088401C80B2E0802189884227D1690093
:1082C0006918C91CC8B200F005F920E0E07A00285E
:1082D0001DDD207B401CC0B22073E17A884216DB92
:1082E0000020207369006918491CC8B200F0F2F838
:1082F0000DE0A07A012807D10020A072690069185A
:10830000891CC8B200F0E6F80020E080207370BD40
:108310004802002070B50546280131494418284616
:10832000FCF723FB00283FD02079052802DA05203E
:10833000207154E020790A2803DA2079401C20714A
:108340004DE0A07A002807D10120A07269006918C9
:10835000491CC8B200F0BEF8208900283FDDE08843
:10836000218988420DDAE088401C80B2E0802189B2
:10837000884234D169006918C91CC8B200F0AAF853
:108380002DE0E07A00282ADD207B401CC0B220735B
:10839000E17A884223DB0020207369006918491CB8
:1083A000C8B200F097F81AE02079052802DD052010
:1083B000207111E02079002803D02079401E20711F
:1083C0000AE0A07A012807D10020A072690069188C
:1083D000891CC8B200F07EF80020E080207370BDD8
:1083E000480200200B48807A0A4AD27A904201D192
:1083F000002070470748807A064A115C1046807A50
:10840000401CC0B290720A2801DB0020907208461E
:10841000EFE700005802002010B500F021F800F04E
:1084200001F810BD10B586B0002002900120039025
:108430000320049000240CE0E000084940188088E4
:108440000190E100054A505801A9F9F7BFFF601CEF
:10845000C4B2012CF0DB06B010BD0000C8950008C6
:1084600000210F4A9172D1721173002014E0C821CB
:1084700002010C4BD218118102210201D218117194
:1084800000210201D21891720201D218D1720201A8
:10849000D2181173411CC8B20128E8DB70470000F4
:1084A000580200204802002010B5002404E02046B5
:1084B000FFF730FF601CC4B2012CF8DB10BD10B513
:1084C000002404E02046FFF7D7FE601CC4B2012C54
:1084D000F8DB10BD0649C97A054A50541146C97ADD
:1084E000491CC9B2D1720A2901DB0021D17270473F
:1084F0005802002000B587B0142102A8F7F7D4FF76
:1085000000BF0E4840690121C90408430B49486176
:10851000084640690121C9040840019000BF00BF1E
:10852000272002900120039000200490059002A9CA
:108530000920C006F9F74AFF07B000BD001002404D
:1085400070B500F089F9054600247DE014206043F1
:108550003F494018C068002800D174E014206043EF
:108560003B494018C068291A14206043384A8018D3
:108570008068814200D266E0142060433449085884
:108580000300FFF711FE07060E0D26272829050018
:1085900000BF0021142060432D4A8018C16036E0DE
:1085A00000BF142060432A490858012801D1012145
:1085B00000E0002114206043254A80180174142033
:1085C0006043114640184168142060438018C16020
:1085D0001DE000BF00BF00BF142060431C494018CD
:1085E000007C0121484014216143194A891808740C
:1085F0001420604311464018C1681420604380185D
:1086000080680918142060438018C16000BF00BF53
:10861000142060430E4A8018017C204600F082F846
:10862000142060430A494018406800280AD01420EA
:10863000604340184068A84204D800220221204626
:1086400000F008F800BF641C042C00DA7EE770BD5F
:10865000BC020020F8B504460D461746042C00DA8B
:1086600004E0262224A12AA0F7F7C2FE00F0F4F8C5
:108670000646142060432A490D50142060434018D8
:10868000C068002803D1142060434018C660002150
:1086900014206043224A80188160032D06D17D2179
:1086A000C90014206043801881601AE0042D07D1AE
:1086B000FF21F53114206043194A8018816010E0D1
:1086C000052D06D1C82114206043154A8018816009
:1086D00007E0062D05D1642114206043104A80185C
:1086E0008160002F01D0F01900E0002014216143C7
:1086F0000B4A89184860F8BD2E2E5C436F72655C8A
:108700005372635C6273705F6C65642E630000007B
:108710006C6564203C204C45445F544F54414C00F0
:10872000BC020020F8B505460E460027002D06D0F5
:10873000012D08D0022D0AD0032D10D10BE0012706
:108740000924E4060CE002270924E40608E02027B7
:108750000924E40604E004270924E40600E0F8BD47
:1087600000BF002E01D0012000E000200246394663
:108770002046F9F732FF00BFF1E7000008B52B48AB
:1087800041424018002849D100BF2948C069012151
:1087900008432749C8610846C069C007C00F009058
:1087A00000BF00BF08460069012108432049086155
:1087B000084600694008400008612F20890488624B
:1087C000084600681B4908400121890708600846DF
:1087D000006808600846406901210843890748612C
:1087E00000BF00BF00BF00BF002001218907086152
:1087F00000BF00200121890748620846C0680121A6
:1088000008438907C8600F20FAF728FA012080077B
:108810000068012108438907086004E0302206A1AE
:108820000CA0F7F7E5FD00BF08BD0000006CDC02FE
:1088300000100240FFFC00002E2E5C436F72655C4E
:108840005372635C6273705F74696D657374616D9C
:10885000702E63003000000010B5F9F7C5FE10BDA2
:1088600010B5012208210748F9F7B7FE6423022258
:10887000A0210548F9F798FF002801D1012010BD7B
:108880000020FCE70004004868020020FEB5044612
:108890000D4616461F4615480078012801D10020D4
:1088A000FEBD012011490870012208211048F9F786
:1088B00094FE6421B0B2E2B2009502910190FF20D3
:1088C00001302040C011A02318430146012309486C
:1088D000FAF746F8002803D1044908700120DFE7C1
:1088E00000200249087000BFDAE700001D000020E8
:1088F0000004004868020020FAF756F9FCF7E0FE91
:10890000FCF76EF8FCF718F9FCF744F9FCF77CFC6F
:10891000FCF732FDFFF780FDFCF732FCFCF766F94F
:108920000122D102AF48F9F758FE6420F9F738FC6C
:10893000F9F702FCAC490860FCF72CF90120FCF7C0
:108940004DFF0120FCF766FFFCF736FFFCF7C8FC83
:10895000FCF772FCFFF7CEFDFFF710FFB0E3F9F76D
:1089600043FEA2490968401A322833D90821092058
:10897000C006F9F729FE002801D1012000E00020FF
:108980000546FCF747FF10210920C006F9F71CFE39
:10899000002801D1012000E000200546FCF71EFF61
:1089A000FFF720FD0446002C14D0012C02D0032C2C
:1089B0000ED106E0012211460920C006F9F70DFE8E
:1089C00007E0002201210920C006F9F706FE00E0B9
:1089D00000BF00BFF9F708FE85490968401A7D21EC
:1089E000C900884275D9FCF7DBFE82490880F9F797
:1089F000FBFD7F4908607F4800880300FFF7D4FB38
:108A000008050B11171D23292F357A4801887A484C
:108A100000F086FC2FE07748018878A000F080FC09
:108A200029E07448018884A000F07AFC23E07148B2
:108A3000018890A000F074FC1DE06E4801889B48FE
:108A400000F06EFC17E06B48018899A000F068FC0C
:108A500011E068480188A4A000F062FC0BE06548C2
:108A60000188B0A000F05CFC05E062480188BCA071
:108A700000F056FC00BF00BF5E480088062805DBFA
:108A8000002201210320FFF7E5FD12E0594800888C
:108A9000032805DB002204210320FFF7DBFD08E0AB
:108AA00054480088032804DA002202210320FFF73B
:108AB000D1FDFCF75BFEB349088008460088012819
:108AC00008D100220421FFF7C5FDAFA000F028FC6B
:108AD00008E020E0002202210120FFF7BBFDB1A049
:108AE00000F01EFCFCF74FFEB649088008460088DF
:108AF000012808D1002201211046FFF7ABFDB2A0EA
:108B000000F00EFC07E0002202211046FFF7A2FD54
:108B1000B4A000F005FCF9F767FDB9490968401AEF
:108B2000B84988425CD900210846FCF7C1FCB64927
:108B3000088008460188B5A000F0F2FB0121002062
:108B4000FCF7B6FCB049088008460188BDA000F0DB
:108B5000E7FB02210020FCF7ABFCAB49088008468C
:108B60000188C5A000F0DCFB03210020FCF7A0FC7D
:108B7000A549088008460188CFA000F0D1FB0F214D
:108B80000020FCF795FCA049088008460188D9A080
:108B900000F0C6FB10210020FCF78AFC9A490880EF
:108BA00008460188E1A000F0BBFB11210020FCF782
:108BB0007FFC9549088008460188ECA000F0B0FBD6
:108BC00012210020FCF774FC8F49088008460188B8
:108BD000F5A000F0A5FB13210020FCF769FCFFE1E4
:108BE0006CE20000000400480000002008000020A3
:108BF000100000201400002054970008544A41310E
:108C000031303120205351492056616C75652069FF
:108C1000733A307825782C636C617373204120534C
:108C200051492028756E737461626C65206C696EA1
:108C30006B29210D0A000000544A413131303120A6
:108C4000205351492056616C75652069733A30781C
:108C500025782C636C61737320422053514920287E
:108C6000756E737461626C65206C696E6B29210D81
:108C70000A000000544A413131303120205351491B
:108C80002056616C75652069733A307825782C63BD
:108C90006C6173732043205351492028676F6F64C0
:108CA000206C696E6B29210D0A00000004970008F2
:108CB000544A413131303120205351492056616CA2
:108CC00075652069733A307825782C636C6173730D
:108CD0002045205351492028676F6F64206C696ECE
:108CE0006B29210D0A000000544A413131303120F6
:108CF000205351492056616C75652069733A30786C
:108D000025782C636C6173732046205351492028C9
:108D10007665727920676F6F64206C696E6B2921AC
:108D20000D0A0000544A413131303120205351495D
:108D30002056616C75652069733A307825782C630C
:108D40006C617373204720535149202876657279EE
:108D500020676F6F64206C696E6B29210D0A00001B
:108D6000544A413131303120205351492056616CF1
:108D700075652052656164204572726F72210D0A1B
:108D80000000000016000020544A413131303120EB
:108D900042415345205431206973204C696E6B2148
:108DA0000D0A0000544A41313130312042415345CF
:108DB000205431206973204E6F74204C696E6B21F2
:108DC0000D0A000018000020544A41313130312092
:108DD0004973204D6173746572204D6F6465210D78
:108DE0000A000000544A4131313031204973205388
:108DF0006C617665204D6F6465210D0A00000000EE
:108E00000C0000201027000004000020544A4131CB
:108E10003130312020526567302042617369632010
:108E2000636F6E74726F6C207265676973746572BC
:108E3000202056616C75652069733A307825780D6D
:108E40000A000000544A4131313031202052656718
:108E50003120426173696320737461747573207289
:108E6000656769737465722056616C7565206973F6
:108E70003A307825780D0A00544A4131313031209A
:108E8000205265673220504859206964656E7469C4
:108E90006669636174696F6E207265676973746572
:108EA000722031202056616C75652069733A3078E4
:108EB00025780D0A00000000544A4131313031203C
:108EC000205265673320504859206964656E746983
:108ED0006669636174696F6E207265676973746532
:108EE0007220322056616C75652069733A3078259E
:108EF000780D0A00544A41313130312020526567E3
:108F0000313520457874656E6465642073746174CE
:108F100075732072656769737465722056616C752C
:108F2000652069733A307825780D0A00544A41313A
:108F30003130312020526567313620504859206940
:108F400064656E74696669636174696F6E207265C9
:108F500067697374657220332056616C756520698A
:108F6000733A307825780D0A00000000544A4131E8
:108F70003130312020526567313720457874656E75
:108F800064656420636F6E74726F6C2072656769CC
:108F9000737465722056616C75652069733A307818
:108FA00025780D0A00000000544A4131313031204B
:108FB00020526567313820436F6E6669677572614C
:108FC00074696F6E207265676973746572203120F1
:108FD00056616C75652069733A307825780D0A0002
:108FE000384908800846018837A000F099F9142113
:108FF0000020FCF75DFA334908800846018840A04C
:1090000000F08EF915210020FCF752FA2D49088056
:10901000084601884AA000F083F916210020FCF7D9
:1090200047FA284908800846018854A000F078F9DA
:1090300017210020FCF73CFA2249088008460188E5
:109040005DA000F06DF918210020FCF731FA1D49F0
:1090500008800846018868A000F062F91921002004
:10906000FCF726FA174908800846018870A000F02E
:1090700057F91A210020FCF71BFA1249088008460C
:10908000018879A000F04CF91B210020FCF710FAB0
:109090000C4908800846018882A000F041F91C2193
:1090A0000020FCF705FA07490880084601888DA0D2
:1090B00000F036F9F9F798FA98490860FFF740FA96
:1090C0004DE4000004000020544A41313130312089
:1090D00020526567313920436F6E6669677572612A
:1090E00074696F6E207265676973746572203220CF
:1090F00056616C75652069733A307825780D0A00E1
:10910000544A41313130312020526567323020538A
:10911000796D626F6C206572726F7220636F756E0D
:109120007465722072656769737465722056616C2C
:1091300075652069733A307825780D0A00000000C3
:10914000544A413131303120205265673231204953
:109150006E7465727275707420736F7572636520BA
:1091600072656769737465722056616C75652069F4
:10917000733A307825780D0A00000000544A4131D6
:10918000313031202052656720323220496E7465BB
:10919000727275707420656E61626C6520726567AD
:1091A00069737465720956616C75652069733A302C
:1091B0007825780D0A000000544A413131303120C1
:1091C00020526567323320436F6D6D756E69636140
:1091D00074696F6E2073746174757320726567694A
:1091E000737465722056616C75652069733A3078C6
:1091F00025780D0A00000000544A413131303120F9
:109200002052656732342047656E6572616C207349
:109210007461747573207265676973746572205622
:10922000616C75652069733A307825780D0A000005
:10923000544A413131303120205265673235204562
:10924000787465726E616C207374617475732072CA
:10925000656769737465722056616C756520697302
:109260003A307825780D0A00544A413131303120A6
:10927000205265673236204C696E6B206661696CDE
:1092800020636F756E7465722072656769737465AB
:109290002056616C75652069733A307825780D0A1F
:1092A00000000000544A41313130312020526567BE
:1092B000323720436F6D6D6F6E20636F6E66696726
:1092C00075726174696F6E20726567697374657217
:1092D0002056616C75652069733A307825780D0ADF
:1092E00000000000544A413131303120205265677E
:1092F000323820436F6E66696775726174696F6E8C
:1093000020726567697374657220332056616C75CD
:10931000652069733A307825780D0A000C0000202A
:109320000FB438B505A80090012189020748009BB9
:10933000049AF7F741F8044600200090A1B20348D0
:10934000F8F7E8FC38BC08BC04B01847D00B002084
:1093500010B500290AD00878002807D005487844BD
:10936000F8F714FC002801D0002010BD0248784412
:1093700010BD00005A0400005204000010B500297E
:109380000AD00878002807D005487844F8F7FEFB93
:10939000002801D0002010BD0248784410BD000014
:1093A0004A0400004204000003B4024878448446A2
:1093B00003BC6047C37AFFFF03B402487844844685
:1093C00003BC60472D7DFFFF000021104220633069
:1093D0008440A550C660E770088129914AA16BB10D
:1093E0008CC1ADD1CEE1EFF13112100273325222B5
:1093F000B5529442F772D662399318837BB35AA35D
:10940000BDD39CC3FFF3DEE3622443342004011484
:10941000E664C774A44485546AA54BB528850995AC
:10942000EEE5CFF5ACC58DD5533672261116300654
:10943000D776F6669556B4465BB77AA719973887FC
:10944000DFF7FEE79DD7BCC7C448E5588668A77814
:109450004008611802282338CCC9EDD98EE9AFF94C
:10946000488969990AA92BB9F55AD44AB77A966AF4
:10947000711A500A333A122AFDDBDCCBBFFB9EEB9C
:10948000799B588B3BBB1AABA66C877CE44CC55CC4
:10949000222C033C600C411CAEED8FFDECCDCDDDEC
:1094A0002AAD0BBD688D499D977EB66ED55EF44E94
:1094B000133E322E511E700E9FFFBEEFDDDFFCCF3C
:1094C0001BBF3AAF599F788F8891A981CAB1EBA190
:1094D0000CD12DC14EF16FE18010A100C230E3200C
:1094E0000450254046706760B9839893FBA3DAB3B4
:1094F0003DC31CD37FE35EF3B1029012F322D2325C
:109500003542145277625672EAB5CBA5A895898583
:109510006EF54FE52CD50DC5E234C324A0148104AB
:109520006674476424540544DBA7FAB79987B89753
:109530005FE77EF71DC73CD7D326F2369106B016FB
:1095400057667676154634564CD96DC90EF92FE913
:10955000C899E9898AB9ABA944586548067827684B
:10956000C018E1088238A3287DCB5CDB3FEB1EFBF3
:10957000F98BD89BBBAB9ABB754A545A376A167A9B
:10958000F10AD01AB32A923A2EFD0FED6CDD4DCDC3
:10959000AABD8BADE89DC98D267C076C645C454CEB
:1095A000A23C832CE01CC10C1FEF3EFF5DCF7CDF93
:1095B0009BAFBABFD98FF89F176E367E554E745E3B
:1095C000932EB23ED10EF01E0004004801000000B0
:1095D00002030405060708090A0B0C0D0E0F1010F4
:1095E0000102030405060708090A0B0C0D0E0F10F3
:1095F0000000000000000000010203040607080943
:109600000000000001020304000000000000000050
:1096100030313233343536373839414243444546A8
:1096200040305800303132333435363738396162A2
:1096300063646566403078000400000800000000A4
:1096400000000002000100001030313233343536A2
:10965000373839616263646566787000303132335F
:109660003435363738394142434445465850000076
:1096700002400000000000A00000000005400000C3
:10968000000000C8000000000C4000000000409CEA
:1096900000000000194000000020BCBE00000000D7
:1096A00034400000BFC91B8E00000004B54000001C
:1096B000504BCFD06607E2CF010000006C410000A4
:1096C0003E8251AADFEEA73401000000D94200001B
:1096D000DCB5A0E23A301F97FFFFFFFFB445000062
:1096E000FD25A0C8E9A3C14FFFFFFFFFFF3F00001A
:1096F0000000008000000000FF3F0000000000802C
:1097000000000000544A413131303120205351498A
:109710002056616C75652069733A307825782C6322
:109720006C6173732044205351492028676F6F6424
:10973000206C696E6B3B20626974206572726F7277
:109740002072617465203C2031652D313029210D56
:109750000A000000544A4131313031202053514930
:109760002056616C75652069733A307825782C77BE
:109770006F727365207468616E20636C617373200F
:10978000412053514928756E737461626C65206C79
:10979000696E6B29210D0A00E49800080000002082
:1097A000B4010000141C0008A8990008B4010020AE
:1097B000B4190000040100081C0000004300000070
:1097C000F8FFFFFF0C0000000E0000000F0000007B
:1097D0002E0000001001000043000000F8FFFFFF12
:1097E00000404040404040404040414141414140B4
:1097F0004040404040404040404040404040404069
:1098000040050202020202020202020202020202F7
:1098100002202020202020202020200202020202FC
:109820000202909090909090101010101010101054
:109830001010101010101010101010100202020260
:1098400002028888888888880808080808080808A4
:1098500008080808080808080808080802020202A0
:1098600040000000000000000000000000000000B8
:1098700000000000000000000000000000000000E8
:1098800000000000000000000000000000000000D8
:1098900000000000000000000000000000000000C8
:1098A00000000000000000000000000000000000B8
:1098B00000000000000000000000000000000000A8
:1098C0000000000000000000000000000000000098
:1098D0000000000000000000000000000000000088
:1098E00000000000012813255E1B086D041A7D048A
:1098F0001AA9041AE90413F15D1B083508131201B3
:10990000140202021640830440572602010203019A
:109910000722040309041A0313B51C1B08B1041A17
:109920006B041AD90441320419432153127A130AE1
:109930000632022A401413FD591B0811044B5B5BCD
:109940002C1A750C134D581B08C904C11ADD181ABE
:10995000CD041AED041ABD041C0902439B111CC05E
:1099600032095E1B01020B130524161001052401A8
:1099700010090104240202052406170107058203C9
:10998000081C100904D1320A1D070501027B2C07AF
:10999000058107110937442A40072A8107112B093D
:0899A00007440A3B04440000E7
:04000005080000C12E
:00000001FF
